:10665600011900000501013C0200000301FA0400D3
:10666600FA0500030A0A5A0B001E0C00FA0D000375
:106676000E00040F0164100096120132130AFA1478
:10668600010215000217010A1801FA1905321A014A
:106696000A1B01FA1C05321FFFFF20FFFF23011E04
:1066A6002400642A00FA2B00FA2C50782D003D2E87
:1066B60000462F001E30006432507833000034321A
:1066C600FA350164360164370150380A643C0064C7
:1066D6003E003C3F000140FFFF411450420A5A432E
:1066E6000AC84405324500B44600FA470178480214
:1066F600034C00FA4EFFFF500606510596520A3229
:10670600530B46540A96560202570546580002593C
:106716000A465A32FA5B010A5C0A325E000A5F00D8
:10672600FE61FFFF64021C66000267FFFF6A0A3C07
:106736006B00006C329673000074000078013279A9
:1067460001327E00FE8100FE84FFFF8500AF8600D9
:10675600018700FA8901088A00009900009D0A96BF
:106766009E00019FFFFFA0FFFFFAFAFA0065006F87
:1067760000790083008D009700A100AC00B600C030
:1067860000CA00D400DE00E800F20058006000688D
:1067960000700078008000880090009800A000A893
:1067A60000B000B800C100C800D000D800DF00E685
:1067B60000EE00F600410047004D00530059005F0F
:1067C6000065006C00710077007D00830089008FF2
:1067D6000095009B00A200A700AC00B200B900C063
:1067E60000C500CA00D200D500DD00E100E700EFD9
:103A39009007C5E0FEA3E0FF90665812692FE49352
:103A4900F599906656E493FC740193FDEFB505076B
:103A5900EEB50403754D009007C51269162275A7C6
:103A69001085F97385FA747E017F00E5741269087F
:103A7900E5732FFF50010E8E5A8F5B900017E0FC03
:103A8900A3E0FDEF2DFDEE3CFC8C5C8D5D2275A75E
:103A99001085F97385FA747E017F00E5741269084F
:103AA900E5732FFF50010E8E5A8F5BAC2CAD2DEFB5
:103AB9002DFDEE3CFC8C5C8D5D22E55DF5FBE55C46
:103AC900F5FCD29322E55DF5E9E55CF5EAD29422AD
:103AD900E55DF5EBE55CF5ECD29122E55DF5EDE50B
:103AE9005CF5EED29222E55DF5FDE55CF5FED28747
:103AF90022E55DF5CEE55CF5CFD29022AE5AAF5BFB
:103B090074068E048F05FF1268F88C5C8D5DAE5AC1
:103B1900AF5B74068E048F05FF1269238C5A8D5B87
:103B2900E55B455A60137406C3955BFFE4955AFE3D
:103B39008E5A8F5B785C12695CE573A85CB80015D6
:103B4900D3955D4010E573C3955DFFE4955CFE8EEA
:103B59005C8F5D8010E573243CC3955DFFE4955C43
:103B6900FE8E5C8F5DAE5CAF5D743B6F4E6006741C
:103B79003C6F4E701AAE5CAF5D743B6F4E7005754D
:103B890073018003757302755D3A755C0080037576
:103B9900730022900095E0B40104C20E8002D20E97
:103BA900900096E0B40104C20F8002D20F9000D3B6
:103BB900E075F0DCA4FFAEF0740A8E048F05FF12E5
:103BC90068F89007BBECF0A3EDF0A20B4016740364
:103BD9008C068D0712690874011200399007B9EE35
:103BE900F0A3EFF07E017F00900091E01269089048
:103BF90000D4E08E048F05FF1268F8740AFF12687A
:103C0900F88D609000DDE075F0DCA4FFAEF0740A79
:103C19008E048F05FF1268F89007BFECF0A3EDF052
:103C29009000DFE060139000DFE0F5F0741684FF88
:103C39007E00EF9007CDF0800674649007CDF09078
:103C490000D5E0900079F090011FE0900063F090BA
:103C590000AEE0900065F09000D7E0900066F0902B
:103C69000083E0900067F0900109E090006CF0900B
:103C7900016DE090006DF090016EE090006EF090A3
:103C8900016FE090006FF0A228B3401690016DE03B
:103C9900700C90016EE0700690016FE06002800286
:103CA900C22874E3900078F09000BEE0B40B087469
:103CB900E3900078F0805A9000BEE0B419129000A9
:103CC900D4E090675D12008CE493900078F0804115
:103CD9009000BEE0B41E129000D4E090677B120001
:103CE9008CE493900078F080289000BEE0B428120C
:103CF9009000D4E09067A512008CE493900078F0CE
:103D0900800F9000BEE0B446089000B5E0900078BE
:103D1900F09000EEE0FE9000BCE06E600A9000BCFE
:103D2900E09000EEF0D22790007CE0FE9000BBE02E
:103D3900B5063390007EE0FE9000D9E0B5062790E5
:103D4900007DE0FE9000E7E0B5061B900080E0FEF4
:103D590090008EE0B5060F90007FE0FE9000C9E06C
:103D69006E7003023F2F9000C9E064036006900063
:103D7900E7E06008740590010AF080067408900174
:103D89000AF090008EE0B4010674009000F4F090FF
:103D9900008EE0B4020674009000D9F090008EE025
:103DA900B4030674009000E6F09000C9E0B403087B
:103DB9009000E7E064026002800674009000E7F07A
:103DC9009000C9E0B403119000D9E0D394014008F0
:103DD9009000E7E064016002800674009000E7F05B
:103DE9009000D9E0D39401401A741890010CF07432
:103DF9000090010DF074009006CFF074009006D089
:103E0900F0803D9000E7E0B401089000C9E0640348
:103E19006002801A740090010CF0741890010DF082
:103E290074009006CFF074009006D0F080127400F0
:103E390090010CF0740090010DF074189006CFF009
:103E49009000BBE0601474079000A2F07400900623
:103E5900D3F074009006D4F0800C74009000A2F0A6
:103E690074079006D3F09000BBE0B4021474089074
:103E790000A3F074009006D7F074009006D8F08083
:103E89000C74009000A3F074089006D7F09000C954
:103E9900E0B402069000E7E0600280147404900622
:103EA900DBF074059006DFF074069006E3F08024D9
:103EB90074009006DBF074009006DCF07400900644
:103EC900DFF074009006E0F074009006E3F07400EF
:103ED9009006E4F0D2279000BBE090007CF09000BF
:103EE900E7E090007DF09000D9E090007EF090002E
:103EF900C9E090007FF090008EE0900080F0900083
:103F09008EE0900064F09000C9E0900068F09000A5
:103F1900E7E0900069F09000BBE090006AF0900043
:103F2900D9E090006BF09000F1E0B4011790002304
:103F3900740FF0A374FFF0900025E4F0A3F074026D
:103F49009000F1F09000F1E0B40341900025E0FE0B
:103F5900A3E0FF900023E0FCA3E0FD126954741074
:103F69001269087408120039EF900075F0EF7006B5
:103F790074FF900075F074009000F1F0900024E057
:103F8900900076F0900023E0900077F0900082E0B6
:103F9900900043F0900043E02414900044F0900016
:103FA90043E02428900045F0900044E0D3943C403D
:103FB9000B900044E0C3943C900044F0900045E02D
:103FC900D3943C400B900045E0C3943C900045F0ED
:103FD900900049E4F0900043E0643B60079000439F
:103FE900E0B43C20900043E0B43B067402900049E1
:103FF900F0900043E0B43C069000497401F0900051
:10400900437401F090004AE4F0900044E0643B609E
:1040190007900044E0B43C20900044E0B43B0674AF
:104029000290004AF0900044E0B43C0690004A74C3
:1040390001F09000447401F090004BE4F0900045C9
:10404900E0643B6007900045E0B43C20900045E007
:10405900B43B06740290004BF0900045E0B43C0676
:1040690090004B7401F09000457401F0900082E0DB
:10407900FE9000E5E02E90004DF09000C0E0B40104
:104089006390004DE0641E600790004DE0B43C066B
:1040990090004DE004F090004DE0641D6007900031
:1040A9004DE0B43B0690004DE014F090004DE0D394
:1040B900943C400B90004DE0C3943C90004DF0902F
:1040C900004DE0D3941E400D90004DE0C3941E9026
:1040D900004EF0800A90004DE0241E90004EF075CD
:1040E900511E807990004DE06414600F90004DE0FE
:1040F9006428600790004DE0B43C0690004DE00450
:10410900F090004DE06413600F90004DE06427606B
:104119000790004DE0B43B0690004DE014F090008C
:104129004DE0D3943C400B90004DE0C3943C90008B
:104139004DF090004DE0D39414400B90004DE0C336
:10414900941490004DF090004DE0D39414400B90DE
:10415900004DE0C3941490004DF07551149000C8BF
:10416900E0900046F0900046E075F01484AFF07ED0
:1041790000EF4E7006900046E004F0900046E0041F
:1041890075F01484AFF07E00EF4E7006900046E0A3
:1041990014F0900046E0B479069000467401F0905E
:1041A9000046E0D3943C400F900046E0C3943C9015
:1041B9000046F0D2218002C221900046E0241490EA
:1041C9000047F0900046E02428900048F09000470E
:1041D900E0D3943C400B900047E0C3943C900047E7
:1041E900F0900048E0D3943C400B900048E0C39421
:1041F9003C900048F022C293C294C291C292C287F5
:10420900C290E5B554EFF5B5E5B554DFF5B5C296FD
:10421900C295C2A0C297C2A2C2A1E5B554BFF5B565
:10422900E5B5547FF5B5E5B554FBF5B5C210755E36
:10423900469000CBE07005756D028003756D0375BE
:10424900550075540090000C74FFF0A374DCF0C2A3
:1042590016C218C21A74C8900037F074C890003B8F
:10426900F074C890003FF0755300755200C20B7589
:104279004600E56FB40903756F0075630090001976
:10428900E4F0A3F0757010C213C214C2159007BBF5
:10429900E0FEA3E0FF74031269087401120039906B
:1042A90007B9EEF0A3EFF0C20275570075560090FA
:1042B9000010E4F0A3F0C229755900755800900068
:1042C9008DE075F032A4FDACF0900021ECF0A3ED87
:1042D900F0C239A22DB39205A22EB39206A22FB332
:1042E9009207A230B39208A231B39209A232B392D3
:1042F9000A2275A71085F97385FA747E017F00E596
:1043090074126908E5732FFF50010E8E5A8F5BAC4A
:104319005CAD5DEF2DFDEE3CFC8C5C8D5D123AC30E
:10432900123ACE123AD99000C9E0B40309123AE41C
:10433900123AEF123AFA75A7002285F97385FA74D1
:104349007E017F00E574126908E5732FFF50010EA5
:104359008E5A8F5B7E017F76900106E0126908AC68
:104369005AAD5BED2FFFEC3EFE8E5C8F5DE55DF592
:10437900EDE55CF5EE900079E4F07412900050F0F0
:104389002285F97385FA747E017F00E57412690844
:10439900E5732FFF50010E8E5A8F5B9007BBE0FC2F
:1043A900A3E0FDEF2DFDEE3CFC8C5C8D5DE55DF53C
:1043B900FDE55CF5FE22056422A2DBB3400890000E
:1043C900D5E0900079F0A2DCB34006C296C295C24E
:1043D900A075D8402285A77275A7109000C9E0641E
:1043E9000360079000E7E0B4022CA2D8B34002C2F0
:1043F90093A2D9B34002C294A2DAB34002C291A2F5
:10440900DBB34002C292A2DCB34002C287A2DDB391
:104419004002C290802DA2D8B3400AC2939000E70F
:10442900E06002C292A2D9B3400AC2949000E7E0C8
:104439006002C287A2DAB3400AC2919000E7E06045
:1044490002C29075D8408572A722900047E4936410
:1044590006600280FE74C89007C1F8E4F0E8A3F092
:1044690075B50075840175A70075FFA090004CE42F
:10447900F075C91075A70F75A1C775A70075D90083
:1044890075CE0C75A70F75F1FE75F2FF75F30775FB
:10449900F47875A4BA75A5FF75A60775AE0075AF52
:1044A900FF75D48175D5FF75D6FF75D7FF75A70040
:1044B90075A20175A14775F80975D80075D90475F4
:1044C900DD0975DE0975D84075A71075D80075D94D
:1044D9000475DA0975DB0975DC0975DD0975DE090D
:1044E90075DF0975D84075A70075E60875E7107579
:1044F900BC0175BE0475BD6C75BE0775BDA075BEE2
:104509000875BD0175BC0075BB1875BC2075BA0866
:1045190075E88075D11375A70F75E10575E200750A
:10452900C7401241FF759700759780740A1268E8B1
:104539007597C0E5975420700280F8758F0275A7AA
:1045490000D2AF75980075A90C75A70F75AB4375A7
:10455900ADFB75AC1E75A71075C91875CA0075CB6A
:104569000075C80475A700758912758E04758C00CD
:10457900758A00C2A9D28C758D00758B00D2ABD219
:104589008E75EF0675D944C29974C8F50975080086
:104599001200E975B5001204E974639007C1F8E4E3
:1045A900F0E8A3F012037574C89007C1F8E4F0E8C5
:1045B900A3F07464F5097508001200E9900064E03D
:1045C90090008EF090008EE0D39403400C7400901C
:1045D900008EF07400900064F0C21E90008EE0908E
:1045E9006267F82828738028A2B44002D21E80206E
:1045F90075A70F75F30F75A700A2A34002D21E80FD
:104609000F75A70F75F31775A700A2A44002D21E54
:0C6267000245EF0245F10245F902460A2B
:10461900A21EB3405F757308E573D3940E5020E56D
:10462900739007C1F8E4F0E8A3F01202447464F54A
:10463900097508001200E97873740126F650D974D7
:10464900029000CAF0900064E090008EF090008E15
:10465900E0906273F8282873801674009000F4F0D3
:10466900800E74009000D9F0800674009000E6F086
:0C62730002466102466302466B0246735D
:10467900D21D805D757301E573D394075020E573EE
:104689009007C1F8E4F0E8A3F01202447464F50954
:104699007508001200E97873740126F650D974017F
:1046A9009000CAF0900064E090008EF090008EE0D7
:1046B90090627FF8282873801674009000F4F080C7
:0F46C9000E74009000D9F0800674009000E6F0A7
:0C627F000246C00246C20246CA0246D2D5
:1046D800C21D900063E090011FF0900064E090001C
:1046E8008EF0900065E09000AEF0900066E09000DB
:1046F800D7F0900067E0900083F0900068E09000A9
:10470800C9F0900069E09000E7F090006AE090003E
:10471800BBF090006BE09000D9F090006CE0900145
:1047280009F090006DE090016DF090006EE090014E
:104738006EF090006FE090016FF090016DE0700CEA
:1047480090016EE0700690016FE060028004C2285C
:104758008002D2289000D4E07006740A9000D4F049
:104768009000B5E0700674E39000B5F09000BBE0EF
:104778000490007CF09000BCE09000EEF0123B9CAE
:10478800E5B54401F5B57406900052F07401900047
:1047980053F07403900055F07405900056F0744679
:1047A800900057F07405900058F07401900059F08B
:1047B800740090005EF07400900061F074FF900047
:1047C80062F07436900158F07430900159F0742DED
:1047D80090015AF0743290015BF0742090015CF003
:1047E800744290015DF0744D90015EF07457900131
:1047F8005FF07420900160F0744D900161F07433A3
:10480800900162F07420900163F07445900164F0A7
:104818007434900165F07436900166F09000F0E011
:10482800900075F09000A7E0900076F09000A8E066
:10483800900077F0A2B6B3920CA2B3B3920DA2A4E3
:10484800B39224A2B4B39225A2A3B3922690007186
:10485800E4F0756F00743A900781F074FD90078258
:10486800F0900072E4F09007BBE0FEA3E0FF740351
:1048780012690874011200399007B9EEF0A3EFF03D
:10488800756E01900050E4F0C223756300C211D226
:1048980012C202757100C22BD203C22CD204C22DDF
:1048A800D205C22ED206C22FD207C230D208C231D8
:1048B800D209C232D20AC21FC220C221C222C227D2
:1048C80012009E755F00756B007561007565327525
:1048D8006600756700756800756900756A00900064
:1048E80019E4F0A3F0756C00D2B2D2A4D2B0D2B160
:1048F800D2A3D2A7D2A6D2A5D2B790008DE0D394E6
:10490800FA400674FA90008DF07E017F00900077DF
:10491800E0126908900076E02FFF50010E90002306
:10492800EEF0A3EFF0EFD394FFEE940F4007900062
:1049380023E4F0A3F0900075E0700674FF90007512
:10494800F09000CAE0D39402400674019000CAF0C7
:104958009000CBE07005756D028003756D039000C3
:10496800CCE0D39401400674009000CCF09000D2C3
:10497800E0C3940A5006740A9000D2F09000DCE07C
:10498800700674019000DCF09000DCE0B4FF06745F
:10499800FE9000DCF09000E3E0D394FE400674FE45
:1049A8009000E3F0900109E0D3940240067401906E
:1049B8000109F090011FE0D39401400674019001B1
:1049C8001FF074019000E9F074019000EAF074009F
:1049D8009000F1F0741B90010EF0741990010FF023
:1049E8007400900111F074299006C7F0742A90069B
:1049F800CBF0D29C9000BCE0D394044006740490A1
:104A080000BCF0E570D3941040037570109006C890
:104A1800E0D3940C400674009006C8F09006CCE0F1
:104A2800D3940C400674009006CCF09006D0E0D3E6
:104A3800940C400674009006D0F09006D4E0D3940D
:104A48000C400674009006D4F09006D8E0D3940C7D
:104A5800400674009006D8F09006DCE0D3940C4031
:104A68000674009006DCF09006E0E0D3940C400653
:104A780074009006E0F09006E4E0D3940C400674CD
:104A8800009006E4F0D2EC75CF01A298B34005C2BD
:104A980098120646E54D6006A299B3B34002800518
:104AA800C299120C57E54E64016005E54EB4040244
:104AB80080D5C28E7E107F00E564126908E58D7589
:104AC800F010A4FDACF0EF2DFDEE3CFCE58B75F08D
:104AD8001084FF7E00ED2FFFEC3EFE8E548F55D2E2
:104AE8008E9000AEE060099000AEE0C3943D4002B5
:104AF800805690001B12691690001BE0FEA3E0FF91
:104B080090001DE0FCA3E0FDEFB5053CEEB50438D0
:104B1800B21CA20BB34013A21CB34008E5B5440471
:104B2800F5B58006E5B554FBF5B590001DE0FEA38C
:104B3800E0FF90001FE0FCA3E0FDEF2DFDEE3CFC44
:104B480090001DECF0A3EDF09000BBE06009900030
:104B5800BBE0C394034003024BE7122D96A20BB3AC
:104B68005009900071E0C3942B400280069000A584
:104B7800E0F545E54575F005A4FFAEF09007C3EEF6
:104B8800F0A3EFF0900092E0C395614007E55FC3A2
:104B9800956050079007C3E4F0A3F0AE2EAF2F90B6
:104BA80007C3E0FCA3E0FDEFD39DEE9C4015E5B5FF
:104BB80054EFF5B59000BBE0B40206E5B54420F526
:104BC800B5801C900071E0C394415006E5B54410CF
:104BD800F5B59000BBE0B40206E5B554DFF5B59035
:104BE80000BBE0B40324122EB1AE2EAF2F9007C342
:104BF800E0FCA3E0FDEFD39DEE9C4008E5B5441032
:104C0800F5B58006E5B554EFF5B5900096E0600976
:104C1800A2B3300D01B3B340028039A2B3300D0105
:104C2800B34031A2B3300F01B3401C9000C9E0B4C7
:104C38000306A21FB3B3400280067404900050F02C
:104C4800D21FA20FB3920DA20FB330B301B3400429
:104C5800A20F920DA2B6300C01B350030252C2A2A9
:104C6800B6300C01B350030252C2A2B6300E01B3E3
:104C78005003025133756E009000AEE0B43D13A2AC
:104C88000EB34008E5B554FBF5B58006E5B5440418
:104C9800F5B5055EA210B3B35013AE54AF559000EE
:104CA8000CE0FCA3E0FDEDC39FEC9E4003024E0325
:104CB800E56DB4032EA229B34022E55EB43B03752B
:104CC8006D01E55EC3943B50069000507401F0E519
:104CD8005ED3943B40067402900050F0755E01D29A
:104CE80029805CE56DB40206756D01755E3BE55E75
:104CF800B43B05755E018047900050E07032E55E78
:104D0800C3943B50069000507401F0E55ED3943B89
:104D180040067402900050F0E55EC3943B5002D206
:104D280023E55ED3943B4002D223C296C295C2A02B
:104D38009000CBE0B401051241FF8003755E01AE1F
:104D480056AF57AC54AD55EF2DFDEE3CFC74028CBC
:104D5800068D071200398E568F579000AEE0600915
:104D68009000AEE0C3943D4002804390001BE0FEFB
:104D7800A3E0FF9000AEE08E048F05FF1268F87480
:104D8800018C068D0712003990001FEEF0A3EFF09A
:104D980090001FE0F8A3E090001DC8F0A3C8F090B1
:104DA800001BE4F0A3F0C21CE5B554FBF5B5A2B4B2
:104DB800B34002C225A2A4B34002C224A2A3B340B6
:104DC80002C226A223B34002C223A21FB34006A2F6
:104DD8002192208002B220900096E06012E56D706A
:104DE8000EA21FB35009A220302101B3B3400280A4
:104DF800067405900050F0C21F803AAE56AF57AC0B
:104E080054AD55EF2DFDEE3CFC74018C068D071258
:104E180000398E568F57E56DC39402500DAC54ADD2
:104E28005574B8C39D740B9C400280091241FF74ED
:104E380006900050F0E55EB43B127403900050F009
:104E4800D2239000CBE0B401031241FFAE58AF5912
:104E5800AC54AD55EF2DFDEE3CFC8C588D59AE543D
:104E6800AF55EFD39DEE9C4011900013E0FAA3E0FC
:104E7800FBEBC394E8EA9403400280069000131207
:104E88006916900010E0FEA3E0FFAC54AD55EF2D7D
:104E9800FDEE3CFC900010ECF0A3EDF09000CBE0B0
:104EA800B40118AE54AF55740512690874011200A4
:104EB8003990000CEEF0A3EFF08011AE54AF5574AA
:104EC8000212690890000CEEF0A3EFF0C28E758D07
:104ED80000758B00756400755501755400D28EE518
:104EE8005E240E75F00F84AFF07E00EF4E70759063
:104EF8000010E0F8A3E090000EC8F0A3C8F09000FE
:104F08000EE0FEA3E0FFEF4E600B7C7B7DF31267A3
:104F1800F68E528F53900010E4F0A3F0AE52AF53C8
:104F28007428BE00039F5010E5632FFF50010E74D4
:104F3800011200398E528F538553639000D2E0A836
:104F480052B8000DD395534008E55390004FF080B8
:104F5800099000D2E01490004FF0E56D600675539B
:104F6800007552009000C9E0B40308900046E0655F
:104F78005E6002800BA220B34004D2228002B222DB
:104F8800E55E640B6005E55EB429099000BBE0604E
:104F9800031223D29000C0E0B4011490004DE065E4
:104FA8005E600790004EE0B55E03756F00801E904E
:104FB800004DE0655E601390004DE02414655E606E
:104FC8000990004DE02428B55E03756F00A211B367
:104FD8005006A210B3B34003025088900087E0B493
:104FE8000173900109E0B40214120E2690007AE0D1
:104FF80075F0BEA4FFAEF08E5C8F5D8056E56775D8
:10500800F00A84FF7E0090058112692FE0F55B7538
:105018005A00AE5AAF5B9000ACE012690874648E17
:10502800048F05FF1268F88C5C8D5DE55D900012B9
:10503800F0AE5AAF5B900085E012690874648E0484
:105048008F05FF1268F874BE8C068D071269088EEA
:105058005C8F5D8017900085E075F0BEA4FFAEF010
:105068008E5C8F5D9000ACE0900012F0E561C39417
:10507800CC5006E55D455C700280031242FBD211FC
:10508800E56DB40106E55E64116002800975700182
:105098009000517401F0E56D600302512E9000CE2E
:1050A800E0600D900079E0A852B8000695534002E0
:1050B80080409000CEE0B4021F900043E0655E603F
:1050C8000F900044E0655E6007900045E0B55E0320
:1050D800757003756C00800CC200756C0090001927
:1050E800E4F0A3F0900079E060067409900050F0B5
:1050F8008034900043E0B55E0B75700190005174E8
:1051080001F08022900044E0B55E0B7570017402D6
:10511800900051F08010900045E0B55E097570016F
:105128007403900051F0A20EB3920CA20EB330B6E5
:1051380001B350030252C2756E019000AEE0B43D57
:1051480013A20EB34008E5B54404F5B58006E5B5ED
:1051580054FBF5B5E5B54401F5B5742B900071F035
:10516800A20E920CE55ED3944A4014D210E55ED3A9
:105178009485400B7404900050F0D223755E4690DD
:1051880000D6E0B40107E56AC3941440028009120E
:1051980041FF7413900050F0A22B300301B3501755
:1051A800A22BB34008E5B54408F5B58006E5B5542B
:1051B800F7F5B5A22B9203A22C300401B35017A225
:1051C8002CB34008E5B54402F5B58006E5B554FDB5
:1051D800F5B5A22C9204A22D300501B3500FA22DD3
:1051E800B34004D2978002C297A22D9205A22E3016
:1051F8000601B35017A22EB34008E5B54410F5B523
:105208008006E5B554EFF5B5A22E9206A22F300719
:1052180001B35017A22FB34008E5B54420F5B58077
:1052280006E5B554DFF5B5A22F9207A23030080184
:10523800B3500FA230B34004D2928002C292A2307F
:105248009208A231300901B3500FA231B34004D201
:10525800878002C287A2319209A232300A01B35074
:105268000FA232B34004D2908002C290A232920AB6
:10527800E56AC394415009740E900050F01241FF42
:10528800900058E0FE900054E0C39E4009900054FE
:10529800E0D39408400974FB900050F01241FF904D
:1052A800005DE0601590005DE0FE900057E06E60E4
:1052B8000974FE900050F01241FFA223B34006C2C9
:1052C80096C295C2A0900106E0600CAE52AF53742E
:1052D80014BE00059F4002804890008EE090628BCB
:1052E800F8282873803BA2B4B35005A225B3400226
:1052F8008005124343D2258028A2A3B35005A226D5
:10530800B340028005124343D2268015A2A4B350AD
:1053180005A224B340028005124343D224800280B0
:015328000084
:10628B000252EC0252EE0253010253140253270244
:02629B00532985
:10532900A213B3B35008900046E0655E60030253D0
:10533900BEA201B35006A200B3B34002807190002F
:10534900C9E0B40343123A67A20BB34021A222B3C6
:105359004005123AC38003123AE49000E7E0B40131
:105369000BA202B34004D2A18002C2A18018123A52
:10537900C3123AE49000E7E0B4010BA202B340047F
:10538900D2A18002C2A180249000E7E0C394025018
:105399000F123A67123AC3A202B34002D292800CAA
:1053A900123A67123AC3123A97123AE475A700C241
:1053B90013D214D215A214B3B35008900047E06574
:1053C9005E6003025453A201B35006A200B3B34076
:1053D9000280719000C9E0B40343123A67A20BB38B
:1053E9004021A222B34005123ACE8003123AEF902F
:1053F90000E7E0B4010BA202B34004D2A18002C2CB
:10540900A18018123ACE123AEF9000E7E0B4010BEE
:10541900A202B34004D2A18002C2A180249000E775
:10542900E0C39402500F123A67123ACEA202B34077
:1054390002D287800C123A67123ACE123A97123A80
:10544900EF75A700D213C214D215A215B3B3500831
:10545900900048E0655E60030254E8A201B350067B
:10546900A200B3B3400280719000C9E0B4034312B3
:105479003A67A20BB34021A222B34005123AD98060
:1054890003123AFA9000E7E0B4010BA202B3400418
:10549900D2A18002C2A18018123AD9123AFA900018
:1054A900E7E0B4010BA202B34004D2A18002C2A179
:1054B90080249000E7E0C39402500F123A67123A31
:1054C900D9A202B34002D290800C123A67123AD99B
:1054D900123A97123AFA75A700D213D214C215E5F7
:0F54E9007090629DF82828730259E69000BCE08D
:06629D000254F10254F46A
:1054F8009062D0F8282873121EAE8012121EAE8059
:0E5508000D121F388008121FE48003121FE4EA
:0F62D0000254FF02550402550902550E025513E0
:105516007570020259E6122110122227A239B340F1
:10552600229000B0E0F56C900081E0256CFE9000C2
:105536004FE075F01E84FC7F00EE2CF5367410905B
:105546000050F09007B9E0FEA3E0FF740A12690864
:1055560090000EE0FCA3E0FD74098F02FF1268F8CC
:105566008D078C038E048A058B061267F69007BD9D
:10557600EEF0A3EFF074F0BE00039F500B74F090B2
:1055860007BDF8E4F0E8A3F0E53670037536019040
:1055960007BDE0FEA3E0FFE5362FFF50010E9007A2
:0D55A600BDEEF0A3EFF0757003900051E032
:0362A30002551C85
:1055B3009062DFF82828738019A23A400375700AB5
:1055C3008010A23A400375700B8007A23A4003751E
:0255D300700C5A
:0C62DF000255BA0255BC0255C50255CE4E
:1055D5000259E69006C8E060031224EA900107E04C
:1055E500B40114900108E0A852B80004955350077F
:1055F500E55FC39560400280097415900050F00284
:1056050056889000BCE0D39402403F900090E0247F
:1056150003A852B8000495535009900092E0D39521
:105625006150028008D2017408900050F0900090FB
:10563500E0A852B80005D39553500B900092E02492
:1056450003C395615002C2018039900090E02403A4
:10565500A852B8000495535007E55FC39560400212
:105665008008D2017408900050F0900090E0A85294
:10567500B80005D395535009E560240FC3955F50D5
:1056850002C2019000D6E07007E56AC39414400297
:105695008002D201A2014005757004800A75701060
:1056A500900019E4F0A3F0A20BB34029E56775F06B
:1056B5000A84FF7E0090058112692FE0C39469502A
:1056C50005122407800F9007BBE0F8A3E09007B907
:0C56D500C8F0A3C8F00259E69000BCE049
:0662A6000255D80256DD8E
:1056E1009062EBF8282873120F108012120F1080AD
:0E56F1000D1210BE800812117080031211708D
:0F62EB000256E80256ED0256F20256F70256FC32
:1056FF009006CCE060031225C67570050259E612BC
:10570F0012B07570069006D0E060031226B69006B0
:10571F00D4E060031227920259E6900012E060066F
:10572F00A20BB3B34002801D900012E02529FFAEFB
:10573F002850010E8E288F29E55ED39414500690C1
:10574F000012E014F01214F67570079006D8E0609E
:10575F000312286E9006DCE0600312294A0259E614
:10576F00900109E0B40203120E9E1218F57570082D
:10577F009006E0E06003122A269006E4E060031230
:10578F002B020259E6121CB1A213B35005A214B397
:10579F0040028006D213D214D2157570100259E64A
:1057AF000259E6900039E0C394465008C2967446F9
:1057BF00900039F0900049E0B4011DE5362406F55C
:1057CF00369007BDE0FEA3E0FF74062FFF50010ED9
:1057DF009007BDEEF0A3EFF0900049E0B4021DE595
:1057EF0036240CF5369007BDE0FEA3E0FF740C2FB6
:1057FF00FF50010E9007BDEEF0A3EFF085365B75FD
:10580F005A00900043E0F573123B05E55D900039B7
:10581F00F0900006E55AF0A3E55BF0E57390003ACF
:10582F00F0C2179007BDE0F55AA3E0F55B90004377
:10583F00E0F573123B05E55D900037F0900000E551
:10584F005AF0A3E55BF0E573900038F0C216E56DF2
:10585F00B4010575700B80037570030259E6900053
:10586F003DE0C394465008C295744690003DF090B9
:10587F00004AE0B4011DE5362406F5369007BDE079
:10588F00FEA3E0FF74062FFF50010E9007BDEEF050
:10589F00A3EFF090004AE0B4021DE536240CF53674
:1058AF009007BDE0FEA3E0FF740C2FFF50010E9098
:1058BF0007BDEEF0A3EFF085365B755A00900044FC
:1058CF00E0F573123B05E55D90003DF0900008E5B3
:1058DF005AF0A3E55BF0E57390003EF0C219900714
:1058EF00BDE0F55AA3E0F55B900044E0F573123B81
:1058FF0005E55D90003BF0900002E55AF0A3E55BF3
:10590F00F0E57390003CF0C218E56DB401057570B9
:10591F000C80037570030259E6900041E0C3944672
:10592F005008C2A07446900041F090004BE0B401C3
:10593F001DE5362406F5369007BDE0FEA3E0FF74A3
:10594F00062FFF50010E9007BDEEF0A3EFF0900071
:10595F004BE0B4021DE536240CF5369007BDE0FE92
:10596F00A3E0FF740C2FFF50010E9007BDEEF0A3C4
:10597F00EFF085365B755A00900045E0F573123BEA
:10598F0005E55D900041F090000AE55AF0A3E55B54
:10599F00F0E573900042F0C21B9007BDE0F55AA3EB
:1059AF00E0F55B900045E0F573123B05E55D900077
:1059BF003FF0900004E55AF0A3E55BF0E57390002B
:1059CF0040F0C21AE56DB40103756D007570038068
:0759DF000680048002800035
:1062AC0002570E02572902576F0257940257AF023A
:1062BC0057B202586D0259280259E00259E20259AC
:0462CC00E40259E6A9
:1059E600900037E0B55E028003025A88A216407224
:1059F600900000E0FEA3E0FFEF4E6021AE56AF57E9
:105A0600900000E0FCA3E0FD12000374068E048FF4
:105A160005FF1268F8900000ECF0A3EDF090003856
:105A2600E0601A900000E0FEA3E0FFAC56AD57EF31
:105A36002DFDEE3CFC900000ECF0A3EDF09000385C
:105A4600E0D39401401A900000E0FEA3E0FFAC56BC
:105A5600AD57EF2DFDEE3CFC900000ECF0A3EDF011
:105A6600D216AE54AF55900000E0FCA3E0FDEFC3A4
:105A76009DEE9C400D12438AD296C21674C89000C1
:105A860037F0A216B3B35007900037E0B55E028038
:105A96000D12438AD29674C8900037F0C216900051
:105AA60039E0B55E028003025B43A21740729000A4
:105AB60006E0FEA3E0FFEF4E6021AE56AF57900022
:105AC60006E0FCA3E0FD12000374068E048F05FFBA
:105AD6001268F8900006ECF0A3EDF090003AE06052
:105AE6001A900006E0FEA3E0FFAC56AD57EF2DFD81
:105AF600EE3CFC900006ECF0A3EDF090003AE0D30B
:105B06009401401A900006E0FEA3E0FFAC56AD57A4
:105B1600EF2DFDEE3CFC900006ECF0A3EDF0D21765
:105B2600AE54AF55900006E0FCA3E0FDEFC39DEE3A
:105B36009C400AC2967446900039F0C217A217B369
:105B4600B35007900039E0B55E02800AC2967446EB
:105B5600900039F0C21790003BE0B55E0280030268
:105B66005BFEA2184072900002E0FEA3E0FFEF4E3B
:105B76006021AE56AF57900002E0FCA3E0FD120094
:105B86000374068E048F05FF1268F8900002ECF08D
:105B9600A3EDF090003CE0601A900002E0FEA3E066
:105BA600FFAC56AD57EF2DFDEE3CFC900002ECF03D
:105BB600A3EDF090003CE0D39401401A900002E07F
:105BC600FEA3E0FFAC56AD57EF2DFDEE3CFC90007A
:105BD60002ECF0A3EDF0D218AE54AF55900002E0FF
:105BE600FCA3E0FDEFC39DEE9C400D12438AD295C7
:105BF600C21874C890003BF0A218B3B350079000C7
:105C06003BE0B55E02800D12438AD29574C89000BF
:105C16003BF0C21890003DE0B55E028003025CB91D
:105C2600A2194072900008E0FEA3E0FFEF4E60214B
:105C3600AE56AF57900008E0FCA3E0FD12000374D7
:105C4600068E048F05FF1268F8900008ECF0A3EDAD
:105C5600F090003EE0601A900008E0FEA3E0FFAC82
:105C660056AD57EF2DFDEE3CFC900008ECF0A3ED91
:105C7600F090003EE0D39401401A900008E0FEA3A5
:105C8600E0FFAC56AD57EF2DFDEE3CFC900008EC66
:105C9600F0A3EDF0D219AE54AF55900008E0FCA386
:105CA600E0FDEFC39DEE9C400AC295744690003D10
:105CB600F0C219A219B3B3500790003DE0B55E02D9
:105CC600800AC295744690003DF0C21990003FE0EC
:105CD600B55E028003025D74A21A4072900004E071
:105CE600FEA3E0FFEF4E6021AE56AF57900004E0F2
:105CF600FCA3E0FD12000374068E048F05FF1268F4
:105D0600F8900004ECF0A3EDF0900040E0601A90EB
:105D16000004E0FEA3E0FFAC56AD57EF2DFDEE3CD0
:105D2600FC900004ECF0A3EDF0900040E0D3940169
:105D3600401A900004E0FEA3E0FFAC56AD57EF2DED
:105D4600FDEE3CFC900004ECF0A3EDF0D21AAE544C
:105D5600AF55900004E0FCA3E0FDEFC39DEE9C4030
:105D66000D12438AD2A0C21A74C890003FF0A21A3C
:105D7600B3B3500790003FE0B55E02800D12438A30
:105D8600D2A074C890003FF0C21A900041E0B55E00
:105D9600028003025E2FA21B407290000AE0FEA35F
:105DA600E0FFEF4E6021AE56AF5790000AE0FCA32D
:105DB600E0FD12000374068E048F05FF1268F8904A
:105DC600000AECF0A3EDF0900042E0601A90000AA1
:105DD600E0FEA3E0FFAC56AD57EF2DFDEE3CFC9088
:105DE600000AECF0A3EDF0900042E0D39401401AD3
:105DF60090000AE0FEA3E0FFAC56AD57EF2DFDEE96
:105E06003CFC90000AECF0A3EDF0D21BAE54AF556B
:105E160090000AE0FCA3E0FDEFC39DEE9C400AC2A1
:105E2600A07446900041F0C21BA21BB3B35007906A
:105E36000041E0B55E02800AC2A07446900041F0BF
:105E4600C21B9000D9E0B402028003025F64900096
:105E560073E0D395665064900073E0F4042566FE03
:105E66009000DCE08E00F5F0E884FF7E008F73EF93
:105E7600C39410500CEF8573F0A4FDACF08D7380C5
:105E8600037573FF900073E0D39573400B90007316
:105E9600E0C39573F57180037571009000F7E0D348
:105EA600957140069000F7E0F5719000F8E0C39513
:105EB6007150069000F8E0F5718071900073E0C3B0
:105EC6009566FE9000DCE08E00F5F0E884FF7E002B
:105ED6008F73EFC39410500CEF8573F0A4FDACF0F4
:105EE6008D7380037573FF85735B755A009000731D
:105EF600E0255BFFAE5A50010E8E5A8F5B74FFBED3
:105F06000009D39F4005855B7180037571FF900082
:105F1600F7E0D3957140069000F7E0F5719000F830
:105F2600E0C3957150069000F8E0F571A20BB3B38B
:105F3600500D900074E0FE9000E4E0D39E50028085
:105F46000A7407900050F0C2A2801375A710E5CD21
:105F5600C395714004C2A28002D2A275A700900028
:105F6600FEE0A852B80004955350179000FDE0A833
:105F760052B8000ED3955340099000FFE0D39561C7
:105F86004002802375A710E5CDC394805008E5B57F
:105F96004480F5B58006E5B5547FF5B5E5B554BF43
:105FA600F5B575A700802175A710E5CDC39480507F
:105FB60008E5B54440F5B58006E5B554BFF5B5E549
:105FC600B5547FF5B575A700900101E0A852B80059
:105FD6000495535017900100E0A852B8000ED395CF
:105FE600534009900102E0D395614002801775A7DE
:105FF60010E5CDC394805004D2A18002C2A1C2A2F2
:1060060075A700801575A710E5CDC394805004D2FE
:10601600A28002C2A2C2A175A700E56FC39409506F
:106026000AA2EDB34005C2ED123050AE54AF55741E
:1060360010C39F74279E400C900072E0C3945A4090
:1060460003026264A210B340091241FF7406900075
:1060560050F0A21EB34008E5B54404F5B58006E548
:10606600B554FBF5B5A212B3500EE561D394334097
:1060760007E561C394CC40028041900109E0B40277
:1060860014120E2690007AE075F050A4FFAEF08E42
:106096005C8F5D800F900085E075F050A4FFAEF038
:1060A6008E5C8F5DE55D455C6011E5B54401F5B537
:1060B600742B900071F01242FBD212900072E0D362
:1060C60094014007E561C3941A40028002C212900F
:1060D60006C8E060031224EAA22B300301B350176E
:1060E600A22BB34008E5B54408F5B58006E5B554DE
:1060F600F7F5B5A22B92039006CCE060031225C6F5
:10610600A22C300401B35017A22CB34008E5B544C5
:1061160002F5B58006E5B554FDF5B5A22C920490BE
:1061260006D0E060031226B6A22D300501B3500F4B
:10613600A22DB34004D2978002C297A22D92059059
:1061460006D4E06003122792A22E300601B3501740
:10615600A22EB34008E5B54410F5B58006E5B55462
:10616600EFF5B5A22E92069006D8E0600312286ECF
:10617600A22F300701B35017A22FB34008E5B5444C
:1061860020F5B58006E5B554DFF5B5A22F92079048
:1061960006DCE0600312294AA230300801B3500F32
:1061A600A230B34004D2928002C292A230920890EA
:1061B60006E0E06003122A26A231300901B3500F2F
:1061C600A231B34004D2878002C287A231920990DD
:1061D60006E4E06003122B02A232300A01B3500F2C
:1061E600A232B34004D2908002C290A232920A90A8
:1061F6000072E0C3945A5010E56FB409099000721A
:10620600E004F0756F00803BE56FB40903756F001D
:10621600755500755400758D00758B00756400907A
:106226000071E0C394415008900071E004F08006CC
:106236007441900071F0900071E0B44106E5B554E8
:10624600FEF5B5900072E0D394014007E56AC39469
:106256004140028009740E900050F01241FF024A3C
:016266008FA8
:1062FA000000010001400160018001A001C001E02D
:10630A0002000300039603B603D603F40400050053
:10631A000512052405360548055A056C057E0590C3
:10632A0005A805C005DE0600061406280646066E00
:10633A0006AE05CF00FF013F015F017F019F01BF4C
:10634A0001DF01FF02FF039503B503D503F303FF42
:10635A0004FF05110523053505470559056B057D1C
:10636A00058F05A705BF05CE05F1061306270645C5
:10637A00066D06AD06ED05DD0FAA0FA50F9F0F9A54
:10638A000F940F8D0F870F800F780F710F680F60B2
:10639A000F570F4E0F450F3B0F300F250F1A0F0ED9
:1063AA000F020EF50EE80EDB0ECC0EBE0EAE0E9FE1
:1063BA000E8E0E7D0E6C0E5A0E470E340E200E0CEB
:1063CA000DF70DE20DCB0DB50D9D0D850D6D0D541F
:1063DA000D3A0D200D050CE90CCE0CB10C940C767F
:1063EA000C580C3A0C1B0BFB0BDB0BBB0B9A0B79F7
:1063FA000B570B350B130AF10ACE0AAB0A870A644C
:10640A000A400A1C09F809D409B0098C096709432A
:10641A00091F08FB08D608B2088E086A084608232E
:10642A0007FF07DC07B9079607730751072F070D00
:10643A0006EC06CA06AA068906690649062A060A53
:10644A0005EC05CD05B0059205750558053C0520F6
:10645A00050504EA04CF04B5049C048204690451C6
:10646A0004390422040B03F403DE03C803B2039DB8
:10647A00038903750361034D033B032803160304D1
:10648A0002F202E102D102C002B002A0029102822B
:10649A000273026502570249023C022F02220216C7
:1064AA00020901FD01F201E601DB01D001C601BBCF
:1064BA0001B101A7019D0194018B0182017901704B
:1064CA000168016001580150014801410139013256
:1064DA00012B0125011E01180111010B010500FF05
:1064EA0000FA0FA60FA00F990F920F8B0F840F7C43
:1064FA000F740F6B0F620F580F4E0F430F380F2C8C
:10650A000F1F0F120F050EF70EE80ED80EC80EB7A2
:10651A000EA50E930E800E6C0E580E420E2C0E1502
:10652A000DFD0DE40DCB0DB10D950D790D5D0D3FF2
:10653A000D200D010CE10CC00C9E0C7C0C590C3585
:10654A000C100BEA0BC40B9E0B760B4F0B260AFDA5
:10655A000AD40AAA0A800A550A2A09FF09D409A8EC
:10656A00097C0950092508F908CD08A10875084AC7
:10657A00081E07F307C8079D07730749072006F790
:10658A0006CE06A6067E06570630060A05E405BFAD
:10659A00059B057705540532051004EF04CE04AEB9
:1065AA00048F047104530435041903FD03E203C77D
:1065BA0003AD0394037B0363034B0334031E0308F5
:1065CA0002F302DE02CA02B602A30291027F026D40
:1065DA00025C024C023C022C021D020E020001F275
:1065EA0001E401D701CA01BE01B101A6019A018FD6
:1065FA000185017A01700166015D0153014A014179
:10660A00013901310129012101190112010B01048A
:10661A0000FD00F700F000EA00E400DE00D900D334
:10662A0000CE00C900C400BF00BA00B500B100AD79
:10663A0000A800A400A0009C009900950091008E7B
:0C664A00008A008700840081007E007B35
:10009E007547009007C5E4F0A3F075310075300088
:1000AE00754D00754E00C236D23774FE9007C7F8F4
:1000BE00E4F0E8A3F074FE9007C9F8E4F0E8A3F0CA
:1000CE0074FE9007D3F0745A9007D4F0745A9007C8
:1000DE00D5F0D238C22AC23AC23522750B00750A43
:1000EE0000AE0AAF0BAC08AD09EDC39FEC9E4016F7
:1000FE0074FF1268E875CF01780B740126F6500470
:10010E0018E436F650DB2290004CE0B4AA1C90079F
:10011E0081E0B43C159007C1E0FEA3E0FFEF4E6016
:10012E0009741EBE0004D39F5003020243755D0086
:10013E00755C0075F8099007C1E0FEA3E0FF740737
:10014E006F4E6006740E6F4E7006743A900781F013
:10015E009007C1E0FEA3E0FF7408BE001ED39F40CF
:10016E001A7E017F089007C1E0FCA3E0FD1DBDFFD4
:10017E00011C1200038E5A8F5B801F9007C1E0FE98
:10018E00A3E0FF740812694C8F048E057E017F0870
:10019E00CDCCCD1200038E5A8F5BAE5CAF5D740C6E
:1001AE00D39F74019E500302023EA2F9B3407EE536
:1001BE005D455C700375A382AE5CAF5D74016F4EDE
:1001CE00700375A300AE5CAF5D74026F4E700D9040
:1001DE0007C2E075F002A4FDACF08DA3AE5CAF5D7E
:1001EE0074036F4E700375A300AE5CAF5D7403BEF7
:1001FE0000039F5013AC5AAD5BED2FFFEC3EFE900B
:10020E00007D12692FE0F5A3AE5CAF5DEFB40B0974
:10021E00EEB4010574141268E8AE5CAF5DEFB40B7A
:10022E0007EEB4010375F80D785C12695C0201A843
:10023E0090004CE4F022755D00755C0075F8099035
:10024E0007C1E0FEA3E0FF7408BE001ED39F401A54
:10025E007E017F089007C1E0FCA3E0FD1DBDFF01FC
:10026E001C1200038E5A8F5B801F9007C1E0FEA305
:10027E00E0FF740812694C8F048E057E017F08CD55
:10028E00CCCD1200038E5A8F5BAE5CAF5D7411D372
:10029E009F74019E5003020374A2F9B3500302032C
:1002AE0071E55D455C700375A3D2AE5CAF5D740104
:1002BE006F4E700375A300AE5CAF5D74026F4E702F
:1002CE000D9007C2E075F002A4FDACF08DA3AE5CFC
:1002DE00AF5D74036F4E700375A300AE5CAF5D74BB
:1002EE00046F4E700375A300AE5CAF5D74056F4E68
:1002FE00700375A300AE5CAF5D74066F4E70037530
:10030E00A300AE5CAF5D74076F4E700375A300AEB5
:10031E005CAF5D74086F4E700375A300AE5CAF5D8D
:10032E007408BE00039F5016AC5AAD5BED2FFFEC68
:10033E003EFE90007812692FE5A3F075A300AE5C27
:10034E00AF5DEFB41009EEB4010574141268E8AE97
:10035E005CAF5DEFB41007EEB4010375F80D785C79
:10036E0012695C02029722755D00755C0075F809D2
:10037E00AE5CAF5D7417BE0004D39F500302044DF4
:10038E00A2F9B3500302044AE55D455C700375A300
:10039E00D2AE5CAF5D74016F4E700375A300AE5CA0
:1003AE00AF5D74026F4E700D9007C2E075F002A43F
:1003BE00FDACF08DA3AE5CAF5D74036F4E70037534
:1003CE00A300AE5CAF5D74046F4E700375A300AEF8
:1003DE005CAF5D74056F4E700375A300AE5CAF5DD0
:1003EE0074066F4E700375A300AE5CAF5D74076F3D
:1003FE004E700375A300AE5CAF5D74086F4E700354
:10040E0075A300AE5CAF5D7408BE00039F500C90E8
:10041E00005A12692FE5A3F075A300AE5CAF5D74B0
:10042E00166F4E700574141268E8AE5CAF5D7416EC
:10043E006F4E700375F80D785C12695C02037E22B4
:10044E0090004CE0B4AB0280030204E8755D0075C9
:10045E005C0075F809AE5CAF5D7412BE007CD39F74
:10046E004078A2F9B34070E55D455C700375A382D8
:10047E00AE5CAF5D74016F4E700375A300AE5CAFE2
:10048E005D74026F4E700D9007C2E075F002A4FD10
:10049E00ACF08DA3AE5CAF5D74036F4E700375A3AD
:1004AE0000AE5CAF5D7403BE00039F500990005F09
:1004BE0012692FE0F5A3AE5CAF5D74116F4E70053F
:1004CE0074141268E8AE5CAF5D74116F4E700375F4
:1004DE00F80D785C12695C020463229007D0E4F098
:1004EE0074649007C1F8E4F0E8A3F012037574C8C1
:1004FE009007C1F8E4F0E8A3F074FF90005AF0748E
:10050E00FF90005BF074FF90005CF074009000545C
:10051E00F074FF90005DF0740090005FF074019035
:10052E000060F0900066E0B4371A900063E090002F
:10053E005AF0900064E090005BF0900065E090004F
:10054E005CF080469007D07401F074659007C1F896
:10055E00E4F0E8A3F012037574C89007C1F8E4F054
:10056E00E8A3F0900066E0B4371A900063E09000C4
:10057E005AF0900064E090005BF0900065E090000F
:10058E005CF0800674029007D0F09007D1E4F0740E
:10059E00669007C1F8E4F0E8A3F012037574C890F2
:1005AE0007C1F8E4F0E8A3F0900065E0B4371290CC
:1005BE000063E0900054F0900064E090005DF080E5
:1005CE00769007D17401F074679007C1F8E4F0E8F3
:1005DE00A3F012037574C89007C1F8E4F0E8A3F015
:1005EE00900065E0B43712900063E0900054F090F4
:1005FE000064E090005DF0803E74029007D1F074CC
:10060E00689007C1F8E4F0E8A3F012037574C8907F
:10061E0007C1F8E4F0E8A3F0900065E0B43712905B
:10062E000063E0900054F0900064E090005DF08074
:10063E000674039007D1F022E54E64046006E59936
:10064E0064FF60028031A2364004D2368027E54E28
:10065E00600874E6254E900050F0E54D600874F089
:10066E00254D900050F0E54EB4010280FE754E000F
:10067E00754D00C2368002C236E54E90384AF828D3
:10068E002873754E00E599B4FF03754D01E599B4D5
:10069E00FE03754D02E599B4FD03754D03E599B45E
:1006AE00FC03754D04E599B4FA03754D05E599B44F
:1006BE00FB06754E011241FFE599B4F906754E041D
:1006CE001241FFE599D394E54007E599C394F040B4
:1006DE0002801685994F754E027E017F00E54FC34D
:1006EE0094E61269088E328F339007C5E4F0A3F0BA
:1006FE00E599D394C44007E599C394E64002802857
:10070E0085994F754E0374E5C3954FF533753200D9
:10071E00AE32AF339062FA1268D7E493F874019355
:10072E009007C5C8F0A3C8F0D299020C569000638A
:10073E00E07005A228B3400280429007C5E0FEA3F8
:10074E00E0FF74FFBE00039F5009EFC39446EE9482
:10075E000640119007C5E0FEA3E0FFEFD3946DEEC7
:10076E00940640139007C5E0FEA3E0FF90008112AF
:10077E00692FE599F0800385997480119007C5E083
:10078E00FEA3E0FF90008112692FE599F09007C556
:10079E001269169007C5E0FEA3E0FFEFB40106EE66
:1007AE00B4070280030209FD900781E0B43C028089
:1007BE00030209FDA22850030208E8C29C900063C0
:1007CE00E090011FF0900064E090008EF0900065C4
:1007DE00E09000AEF0900066E09000D7F0900067D9
:1007EE00E0900083F0900068E09000C9F0900069FE
:1007FE00E09000E7F090006AE09000BBF090006B94
:10080E00E09000D9F090006CE0900109F090006D3E
:10081E00E090016DF090006EE090016EF090006F30
:10082E00E090016FF0123B9C900075E09000F0F0AC
:10083E00900076E09000A7F0900077E09000A8F08E
:10084E0074639007C1F8E4F0E8A3F074AB90004C29
:10085E00F012044E90004CE4F07464F50975080033
:10086E001200E9A21D4039757301E573D394075048
:10087E002DE5739007C1F8E4F0E8A3F074AA900098
:10088E004CF0120115E573C39407500A7464F50910
:10089E007508001200E97873740126F650CC803783
:1008AE00757308E573D3940E502DE5739007C1F858
:1008BE00E4F0E8A3F074AA90004CF0120115E57371
:1008CE00C3940E500A7464F5097508001200E97895
:1008DE0073740126F650CC0209E7C29C90011FE00A
:1008EE00900063F090008EE0900064F09000AEE017
:1008FE00900065F09000D7E0900066F0900083E0E5
:10090E00900067F09000C9E0900068F09000E7E07A
:10091E00900069F09000BBE090006AF09000D9E082
:10092E0090006BF0900109E090006CF07400900064
:10093E006DF0740090006EF0740090006FF07463B0
:10094E009007C1F8E4F0E8A3F074AB90004CF012FD
:10095E00044E90004CE4F07464F509750800120022
:10096E00E9757301E573D394075026E5739007C1BB
:10097E00F8E4F0E8A3F074AA90004CF0120115749C
:10098E0064F5097508001200E97873740126F650B3
:10099E00D3D29C7599FB743C900781F0757308E572
:1009AE0073D3940E5026E5739007C1F8E4F0E8A3D4
:1009BE00F074AA90004CF01201157464F5097508D4
:1009CE00001200E97873740126F650D374C89007AC
:1009DE00C1F8E4F0E8A3F080FE74C89007C1F8E413
:1009EE00F0E8A3F0D29C754E00754D007599FB0290
:1009FE000C569007C5E0FEA3E0FFEF4E70068599FA
:100A0E00317530009007C5E0FEA3E0FF74016F4E14
:100A1E00701BAC30AD31AA32AB33ED2BFBEC3AFA96
:100A2E008A068B0790008112692FE599F09007C511
:100A3E001269169007C5E0FEA3E0FF74026F4E70B8
:100A4E0021AC30AD3174566D4C7006E54F64E660E6
:100A5E000280031241FF123B9C854F99754E007523
:100A6E004D00020C569007C5E0FEA3E0FF900081FA
:100A7E0012692FE599F09007C51269169007C5E027
:100A8E00FEA3E0FFAC32AD338F028E038C068D07D2
:100A9E0090633E1268D7E493F9740193FEEAD39EF5
:100AAE00EB994009854F99754E00754D00020C5615
:100ABE009007C5E0FEA3E0FF90008112692FE59933
:100ACE00F09007C51269169007C5E0FEA3E0FFEF90
:100ADE00B40006EEB401028003020C5690005CE0F6
:100AEE00D394C7400B90005CE0C394C8F550801AB5
:100AFE0090005CE0D39463400B90005CE0C3946480
:100B0E00F550800690005CE0F550E55075F002A4BB
:100B1E00FFAEF08F73EF90008112693AEFFCE0FDAB
:100B2E00EC90008412693AEDFCE0FDEC2DB550021C
:100B3E008003020C470FEF90008112693AE573FFB4
:100B4E00E0FCEF90008512693AECFFE0FCEFC39CED
:100B5E00B550028003020C47E57390008312693A88
:100B6E00E573FFE0FCEF90008612693AECFFE0FCC3
:100B7E00EF2CB550028003020C47E57390008712EC
:100B8E00693AE0C39550900063F0E57390008812C7
:100B9E00693AE0C39550900064F0E57390008912B5
:100BAE00693AE0C39550900065F07400900066F0CD
:100BBE0074FF900067F0E57390008B12693AE0C302
:100BCE009550900068F0E57390008C12693AE0C37E
:100BDE009550900069F0E57390008D12693AE0C36C
:100BEE00955090006AF0E57390008A12693AE0C35E
:100BFE0095509007C1F8E4F0E8A3F074AB90004C68
:100C0E00F012044E7464F5097508001200E990079D
:100C1E00C112691612044E7464F5097508001200AB
:100C2E00E99007C112691612044E7599F97464F5AC
:100C3E00097508001200E980FE7599FF7464F509C4
:080C4E007508001200E980FEA8
:0F384A0002069002073B020A00020A73020ABE3E
:100C560022E54D903859F8282873020D699007C58A
:100C6600E0FEA3E0FF90005212692FE0F59990078D
:100C7600C51269169007C5E0FEA3E0FF74116F4E1A
:100C86007003754D00020D69856E99020D69900716
:100C9600C5E0FEA3E0FF90008112692FE0F599EF11
:100CA600B40107EEB40703754D009007C512691627
:070CB600020D699007C6E082
:0F385900020C60020C63020C8E020C94020CB97C
:100CBD00903A0CF8282873855399020D5E855F993B
:100CCD00020D5E856199020D5E856599020D5E8549
:100CDD006799807D85689980788569998073856A23
:100CED0099806E90001AE0F5998066A237B340079F
:100CFD007599FAC2378041A227B3400575990F80C7
:100D0D00359007D0E0600A9007D0E024DCF599809B
:100D1D00169007D1E0600A9007D1E024DEF59980A6
:100D2D0006900050E0F599900050E4F09007D0E463
:100D3D00F09007D1E4F0C2278017856B998012855A
:100D4D006699800D856C9980087599FC8003754DA9
:010D5D000095
:103A0C00020CC4020CCA020CD0020CD6020CDC0252
:103A1C000CE1020CE6020CEB020CF0020CF8020DAD
:0D3A2C0047020D4C020D51020D56020D5BBC
:0B0D5E009007C51269168003123A3995
:03386800020D66E8
:100D690022E537255BFFAE5A50010E9000811269CA
:100D79002FE0F538E537255BFFAE5A50010E0FBF5E
:100D890000010E90008112692FE0F539853F3BE59E
:100D990038B539058538378041E539D39538401D4F
:100DA900E539C39538853AF0A4FFAEF0E53B8E04EA
:100DB9008F05FF1268F8ED2538F537801DE538C332
:100DC9009539853AF0A4FFAEF0E53B8E048F05FF17
:100DD9001268F8EDF4042538F53722E539D395384A
:100DE900401DE539C39538853AF0A4FFAEF0E53BDF
:100DF9008E048F05FF1268F8ED2538F537801DE55B
:100E090038C39539853AF0A4FFAEF0E53B8E048FDF
:100E190005FF1268F8EDF4042538F53722900087AC
:100E2900E0B40170E56775F00A84FF7E008F37E54D
:100E39006775F00A84ADF07C008D3A753F0A755AE2
:100E490005755B24E537C394115005120D6A8006B8
:100E59009005B6E0F537E53790007AF0E56775F06B
:100E69000A84FF7E008F37E56775F00A84ADF07C50
:100E7900008D3A753F0A755A05755B5AE537C39473
:100E8900115005120D6A80069005ECE0F537E5373B
:100E9900900012F022900087E0B4016AE56775F0CE
:100EA9000A84FF7E008F37E56775F00A84ADF07C10
:100EB900008D3A753F0A755A05755B36E537C39457
:100EC900115005120D6A80069005C8E0F53785377F
:100ED9004BE56775F00A84FF7E008F37E56775F08B
:100EE9000A84ADF07C008D3A753F0A755A05755B29
:100EF90048E537C394115005120D6A80069005DA4A
:100F0900E0F53785374C22E55F75F00484FF7E00F4
:100F19008F37E55F75F00484ADF07C008D3A753F3D
:100F290004755A01755B00E537C3943F5005120DEE
:100F39006A80069001C0E0F5378537297528009049
:100F4900004FE075F020A4FFAEF09000D2E08E04CF
:100F59008F05FF1268F88D379000BAE0D3955F507E
:100F6900030210169000DEE0D3955F4010ED90016A
:100F7900C112693AE0F52B752A000210139000A9F5
:100F8900E0D3955F4043E5379001C112693AE0F536
:100F990038E5379001E112693AE0F5399000DEE071
:100FA900F404255FF53A9000A9E0FE9000DEE0F434
:100FB900042EF53BE538B539058538378003120D20
:100FC900E485372B752A008041E5379001E11269E4
:100FD9003AE0F538E53790020112693AE0F53990BF
:100FE90000A9E0F404255FF53A9000BAE0FE90000C
:100FF900A9E0F4042EF53BE538B539058538378085
:1010090003120DE485372B752A000210BD9000E10B
:10101900E0D3955F5011E53790024112693AE0F546
:101029002B752A000210BD9000AAE0D3955F5043AA
:10103900E53790022112693AE0F538E53790024127
:1010490012693AE0F5399000AAE0F404255FF53A0F
:101059009000E1E0FE9000AAE0F4042EF53BE538AB
:10106900B539058538378003120DE485372B752A84
:10107900008041E53790020112693AE0F538E53719
:1010890090022112693AE0F5399000BAE0F404259A
:101099005FF53A9000AAE0FE9000BAE0F4042EF55C
:1010A9003BE538B539058538378003120DE48537B6
:1010B9002B752A00229000F2E0F53C753F11755A14
:1010C90002755B00AE52AF53E53C75F00FA4FDAC61
:1010D900F0EDD39FEC9E4021E53C8E048F05FF1275
:1010E90068F8ED75F010A4FFAEF0E55F75F01184B6
:1010F900FD7C00ED2FF53D800EE55F75F01184FF55
:101109007E00EF24F0F53D853D37E55F75F01184EC
:10111900AFF07E008F3A120D6A85373EAE52AF535B
:101129009000F2E075F00FA4FDACF0EDD39FEC9EBA
:101139004028755A02755B10853D37120D6A853E48
:1011490038853739AE52AF53E53C8E048F05FF120F
:1011590069238D3A853C3B120DE4853729752800B2
:10116900752B64752A00229000F2E0F53C753F1159
:10117900755A02755B00AE52AF53E53C75F00FA48A
:10118900FDACF0EDD39FEC9E4021E53C8E048F052C
:10119900FF1268F8ED75F010A4FFAEF0E56175F087
:1011A9001184FD7C00ED2FF53D800EE56175F01190
:1011B90084FF7E00EF24F0F53D853D37E56175F04C
:1011C9001184AFF07E008F3A120D6A85373EAE5218
:1011D900AF539000F2E075F00FA4FDACF0EDD39F92
:1011E900EC9E4028755A02755B10853D37120D6AD1
:1011F900853E38853739AE52AF53E53C8E048F05AD
:10120900FF1269238D3A853C3B120DE48537297518
:101219002800E56B6017E56BC394FE50109000E65B
:10122900E0B402099000D4E0D3940B50028017AEC9
:1012390028AF29E56B12690874E78E048F05FF1240
:1012490068F88C288D299000BCE0B40453E55F75DB
:10125900F00484FF7E008F37E55F75F00484ADF0FC
:101269007C008D3A753F04755A01755B00E537C3FB
:10127900943F5005120D6A80069001C0E0F537AE23
:1012890028AF29E53712690874648E048F05FF12A7
:1012990068F8AE28AF29EF2DFDEE3CFC8C288D298E
:1012A900752B64752A0022900087E0B40146E56732
:1012B90075F00A84FF7E008F37E56775F00A84AD03
:1012C900F07C008D3A753F0A755A05755B00E53764
:1012D900C394115005120D6A8006900592E0F53706
:1012E900AE2AAF2BE5372FFF50010E746412694CFB
:1012F9008E2A8F2B900088E0B40146E56875F00AC4
:1013090084FF7E008F37E56875F00A84ADF07C00B4
:101319008D3A753F0A755A05755B6CE537C39411AB
:101329005005120D6A80069005FEE0F537AE2AAF2A
:101339002BE5372FFF50010E746412694C8E2A8FEA
:101349002B900097E0B40249E56AC3944175F00512
:1013590084FF7E008F37E56A75F00584ADF07C0067
:101369008D3A753F05755A06755B00E537C39413C9
:101379005005120D6A8006900694E0F537AE2AAF43
:101389002BE5372FFF50010E746412694C8E2A8F9A
:101399002B9000D9E0B40202800302144FE55F7577
:1013A900F01584FF7E008F37E55F75F01584ADF089
:1013B9007C008D3A753F15755A03755BF4E537C3A3
:1013C900940B5005120D6A8006900480E0F537E50C
:1013D9003775F0FFA4FFAEF09000DAE08E048F05B8
:1013E900FF1268F8ED900073F0E56675F078A4FFD8
:1013F900AEF074FF8E048F05FF1268F88C5A8D5B6E
:1014090074028C068D071200398F37AC5AAD5B74A4
:1014190004FF1269238D3A753F04755A06755B28D6
:10142900E537C3941D5005120D6A80069006C6E083
:10143900F537AE2AAF2BE5372FFF50010E74641232
:10144900694C8E2A8F2B900086E0B4025DE56175A8
:10145900F064A4FFAEF074081200398E5C8F5D74DD
:10146900058E048F05FF1268F88D37AE5CAF5D7489
:10147900058E048F05FF1269238D3A753F05755A4C
:1014890005755BDEE537C394135005120D6A8006B6
:10149900900672E0F537AE2AAF2BE5372FFF5001E2
:1014A9000E746412694C8E2A8F2B9000C8E0703C30
:1014B90090004FE075F00584FF7E008F3790004F54
:1014C900E075F00584ADF07C008D3A753F05755ADD
:1014D90005755BC0E537C3941D5005120D6A80067A
:1014E90090065EE0F537E53790007BF02290008F9B
:1014F900E0B401179007CCE0252BFFAE2A50010E6E
:101509009000E3E012694C8E2A8F2B900107E0B41A
:101519000114900108E0A852B8000495535007E55A
:101529005FC39560400280129000B1E0252BFFAEA9
:101539002A50010E8E2A8F2B802F90008FE0B40342
:1015490016A22AB3B350109007CFE0C39405A8524E
:10155900B800069553400280109000B1E0252BFF9A
:10156900AE2A50010E8E2A8F2B900089E0B4020218
:1015790080030218F490008CE0602FE567D394464D
:101589004028900013E0FEA3E0FF9000C7E075F04B
:1015990003A4FDACF0EFD39DEE9C400E9000EBE070
:1015A900A852B80005D3955350030218F49000BC13
:1015B900E0B40302800302175885615B755A0090F5
:1015C9000093E0A852B800049553500E900094E09F
:1015D900A85AB80005D3955B5003021755E5617504
:1015E900F002A4FFAEF074158E048F05FF1268F89F
:1015F9008C068D0790061112692FFEE0FFEE900010
:101609008BE0FEEF8E0088F0A4FFAEF074648E04C8
:101619008F05FF1268F88C5A8D5B90004FE075F0CA
:1016290018A4FFAEF09000D2E08E048F05FF126877
:10163900F88C068D0790062912692FAE5AAF5BE028
:1016490012690874648E048F05FF1268F88C5A8D2C
:101659005BE565A85AB80077D3955B4072E565C329
:10166900955BFFE4955AFE8E5A8F5B7428BE000382
:101679009F500C755B28755A00740D900050F0AEA0
:101689005AAF5B90008CE012690874288E048F05AC
:10169900FF1268F88C5A8D5BAE28AF29740A8E0444
:1016A9008F05FF1268F88D068C07AC5AAD5BCFCE5B
:1016B900CF120003740A8E048F05FF1268F88C5A42
:1016C9008D5BAE28AF291269548E288F29807DE55C
:1016D90065A85AB80004955B5072AE5AAF5BE565D0
:1016E90012694C8E5A8F5B7428BE00039F500C758B
:1016F9005B28755A00740D900050F0AE5AAF5B909C
:10170900008CE012690874288E048F05FF1268F8AE
:101719008C5A8D5BAE28AF29740A8E048F05FF128F
:1017290068F88D068C07AC5AAD5BCFCECF1200039B
:10173900740A8E048F05FF1268F88C5A8D5BAE28E7
:10174900AF29EF2DFDEE3CFC8C288D290218F49071
:1017590000D4E0855FF0A4FFAEF074051269087447
:10176900071200398E5A8F5B900093E0A852B80097
:101779000495535012900094E075F002A4FDACF06A
:10178900EFC39DEE9C40030218F4E55F75F00B84EE
:10179900FF7E0090061112692FFEE0FFEE90008B8C
:1017A900E0FEEF8E0088F0A4FFAEF074648E048F23
:1017B90005FF1268F88C5A8D5B90004FE075F018A0
:1017C900A4FFAEF09000D2E08E048F05FF1268F8F6
:1017D9008C068D0790062912692FAE5AAF5BE0126D
:1017E900690874648E048F05FF1268F88C5A8D5B42
:1017F900E565A85AB80077D3955B4072E565C3954E
:101809005BFFE4955AFE8E5A8F5B7428BE00039FD6
:10181900500C755B28755A00740D900050F0AE5A43
:10182900AF5B90008CE012690874288E048F05FF65
:101839001268F88C5A8D5BAE28AF29740A8E048F12
:1018490005FF1268F88D068C07AC5AAD5BCFCECF79
:10185900120003740A8E048F05FF1268F88C5A8DE2
:101869005BAE28AF291269548E288F29807DE565E2
:10187900A85AB80004955B5072AE5AAF5BE5651281
:10188900694C8E5A8F5B7428BE00039F500C755BA0
:1018990028755A00740D900050F0AE5AAF5B900055
:1018A9008CE012690874288E048F05FF1268F88C81
:1018B9005A8D5BAE28AF29740A8E048F05FF126812
:1018C900F88D068C07AC5AAD5BCFCECF12000374EE
:1018D9000A8E048F05FF1268F88C5A8D5BAE28AF0B
:1018E90029EF2DFDEE3CFC8C288D29229000E7E0A4
:1018F900B4026AE55F75F00884FF7E008F37E55F03
:1019090075F00884ADF07C008D3A753F08755A0171
:10191900755BE0E537C3943F5005120D6A80069068
:101929000280E0F53785372D752C00AE2CAF2DAC34
:101939002AAD2B12000374648E048F05FF1268F818
:101949008C2C8D2D900084E08C068D07126908740B
:10195900648E048F05FF1268F88C2C8D2DAE28AF8C
:1019690029AC2AAD2B12000374648E048F05FF1273
:1019790068F88C288D29900084E08C068D071269FF
:101989000874648E048F05FF1268F88C288D29A2CB
:101999000B401DAE52AF537405BE00039F5002D2D7
:1019A9000BE561D394CC4008D2017411900050F03A
:1019B9009000E6E0B402089000D4E0640B60028075
:1019C90035AE28AF29E56B12690874E78E048F05D7
:1019D900FF1268F88C288D299000E7E0B40217AE51
:1019E9002CAF2DE56B12690874E78E048F05FF1281
:1019F90068F88C2C8D2D9000A6E05402601B900095
:101A09009DE0A852B80012D39553400DA20BB3B371
:101A19005007E561C3949A40028028AE34AF3590EF
:101A2900009BE075F002A4FDACF0EF2DFDEE3CFC4F
:101A390074022DFD50010CE561BC0007D39D4003E4
:101A4900754301856135753400E5437003021B3820
:101A59009000F9E0C395435003021B2A900109E065
:101A6900C394025076E56775F00A84FF7E009005FD
:101A79008112692FE0F55B755A00AE5AAF5B900091
:101A89009CE012690874648E048F05FF1268F88C53
:101A99005C8D5D9000F9E004C395438C068D0712B7
:101AA90069089000F9E08E048F05FF1268F88C5CD4
:101AB9008D5DAE28AF29EF2DFDEE3CFC8C288D29DC
:101AC9009000E7E0B40212AE2CAF2DAA5CAB5DEF3B
:101AD9002BFBEE3AFA8A2C8B2D80469000F9E00414
:101AE900C39543854BF0A4FFAEF09000F9E08E0456
:101AF9008F05FF1268F88C5C8D5DAE28AF29EF2D3C
:101B0900FDEE3CFC8C288D299000E7E0B40212AE72
:101B19002CAF2DAA5CAB5DEF2BFBEE3AFA8A2C8B2E
:101B29002D05439000F9E0C3954350037543009098
:101B390000A6E05401601B90009AE0A852B8001278
:101B4900D39553400DA20BB3B35007E55FC394CCB3
:101B590040028025900098E075F003A4FFAEF0E5FF
:101B6900402FFF50010E74032FFF50010EE55FBE99
:101B79000007D39F4003754401855F40E544700326
:101B8900021C6B9000FAE0C395445003021C5D905F
:101B99000109E0C394025076E56775F00A84FF7E77
:101BA9000090058112692FE0F55B755A00AE5AAFB6
:101BB9005B900099E012690874648E048F05FF1226
:101BC90068F88C5C8D5D9000FAE004C395448C063E
:101BD9008D071269089000FAE08E048F05FF1268DC
:101BE900F88C5C8D5DAE28AF29EF2DFDEE3CFC8CA9
:101BF900288D299000E7E0B40212AE2CAF2DAA5C23
:101C0900AB5DEF2BFBEE3AFA8A2C8B2D80469000C8
:101C1900FAE004C39544854CF0A4FFAEF09000FAB5
:101C2900E08E048F05FF1268F88C5C8D5DAE28AFDD
:101C390029EF2DFDEE3CFC8C288D299000E7E0B4BE
:101C49000212AE2CAF2DAA5CAB5DEF2BFBEE3AFA7C
:101C59008A2C8B2D05449000FAE0C39544500375F6
:101C690044009000FCE02529FFAE2850010E8E2883
:101C79008F299000ABE0A828B80004952950099055
:101C890000ABE0F5297528009000E7E0B4020D905B
:101C990000ABE0A82CB80006952D40028009900001
:101CA900ABE0F52D752C00229000E7E0B40102802D
:101CB90003021DBCA20BB35003021DBA9000B2E08F
:101CC900B40168AE28AF29AC52AD53120003743C7D
:101CD9008E048F05FF1268F89000C2E0BC00109DC9
:101CE900400D9000C4E0A828B8000495295002D2FC
:101CF90002AE28AF29AC52AD53120003743C8E04D6
:101D09008F05FF1268F89000C2E0C3940ABC001561
:101D1900D39D40119000C4E0C39405A828B80005DC
:101D2900D3952950028002C2028068AE28AF29AC3F
:101D390052AD5312000374788E048F05FF1268F8B0
:101D49009000C2E0BC00109D400D9000C4E0A8289E
:101D5900B8000495295004D2028038AE28AF29ACC6
:101D690052AD5312000374788E048F05FF1268F880
:101D79009000C2E0C3940ABC0015D39D40119000A5
:101D8900C4E0C39405A828B80005D395295002805A
:101D990002C202A202B34019AE28AF299000C3E0E3
:101DA90012690874648E048F05FF1268F88C288DF7
:101DB900298002C202A200B34006A201B3B35009AE
:101DC900900019E4F0A3F08024AE28AF297400D361
:101DD9009F74019E400C900019E528F0A3E529F0B5
:101DE900800B74FF900019F8E4F0E8A3F09000C9A3
:101DF900E0D39402400C9000B4E07006A20BB3B398
:101E09004002801AAE28AF2974021269088E288F01
:101E190029AE2CAF2D74021269088E2C8F2D9000DB
:101E2900B2E0B4011AAE28AF2974021269088E28EB
:101E39008F29AE2CAF2D74021269088E2C8F2DAE0E
:101E490028AF29745E126908740A8E048F05FF127F
:101E590068F88C288D299000E7E0B40217AE2CAF02
:101E69002D745E126908740A8E048F05FF1268F8D2
:101E79008C2C8D2DAE28AF297402BE000AD39F4049
:101E890006752902752800AE2CAF2D7402BE000A12
:101E9900D39F4006752D02752C00900017E528F098
:101EA900A3E529F02290004FE090038112693AE0FE
:101EB900F54175426490004FE0FE9000BDE0D39E6D
:101EC9004037E55F75F00884FF7E008F37E55F7561
:101ED900F00884ADF07C008D3A753F08755A03759A
:101EE9005B96E537C3941F5005120D6A800690046E
:101EF90036E0F5378537428035E55F75F00884FFB0
:101F09007E008F37E55F75F00884ADF07C008D3A6F
:101F1900753F08755A03755BB6E537C3941F5005BD
:101F2900120D6A8006900456E0F5378537422290F3
:101F390000F3E0F53C753F11755A04755B00AE522C
:101F4900AF53E53C75F00FA4FDACF0EDD39FEC9ECB
:101F59004021E53C8E048F05FF1268F8ED75F010FD
:101F6900A4FFAEF0E55F75F01184FD7C00ED2FF55F
:101F79003D800EE55F75F01184FF7E00EF24F0F5DA
:101F89003D853D37E55F75F01184AFF07E008F3AEE
:101F9900120D6A85373EAE52AF539000F3E075F0EB
:101FA9000FA4FDACF0EDD39FEC9E4028755A047543
:101FB9005B10853D37120D6A853E38853739AE523B
:101FC900AF53E53C8E048F05FF1269238D3A853C9A
:101FD9003B120DE4853741754264229000F3E0F528
:101FE9003C753F11755A04755B00AE52AF53E53C21
:101FF90075F00FA4FDACF0EDD39FEC9E4021E53CBC
:102009008E048F05FF1268F8ED75F010A4FFAEF08D
:10201900E56175F01184FD7C00ED2FF53D800EE53D
:102029006175F01184FF7E00EF24F0F53D853D37A1
:10203900E56175F01184AFF07E008F3A120D6A8563
:10204900373EAE52AF539000F3E075F00FA4FDACEC
:10205900F0EDD39FEC9E4028755A04755B10853DC1
:1020690037120D6A853E38853739AE52AF53E53C94
:102079008E048F05FF1269238D3A853C3B120DE4CE
:102089008537417542649000BCE0B4047990004FF3
:10209900E0FE9000BDE0D39E4037E55F75F008840F
:1020A900FF7E008F37E55F75F00884ADF07C008D09
:1020B9003A753F08755A03755B96E537C3941F5007
:1020C90005120D6A8006900436E0F537853742809F
:1020D90035E55F75F00884FF7E008F37E55F75F0A1
:1020E9000884ADF07C008D3A753F08755A03755B1D
:1020F900B6E537C3941F5005120D6A800690045641
:10210900E0F53785374222900087E0B4013BE56767
:1021190075F00A84FF7E008F37E56775F00A84AD94
:10212900F07C008D3A753F0A755A05755B12E537E3
:10213900C394115005120D6A80069005A4E0F53785
:10214900E5422537C39464F542900088E0B4013B29
:10215900E56875F00A84FF7E008F37E56875F00A37
:1021690084ADF07C008D3A753F0A755A05755B7E22
:10217900E537C394115005120D6A8006900610E0E8
:10218900F537E5422537C39464F542E5412542F523
:102199003690008FE0B402109007CBE02536FE9010
:1021A90000E3E0F4042EF5369000E6E0D394014014
:1021B90040E56BC394E7501D74E7C3956BFE900728
:1021C900CDE08E00F5F0E884FF7E008F37E53625F7
:1021D90037F536801CE56BC394E7FE9007CDE08E9A
:1021E90000F5F0E884FF7E008F37E536C39537F5B3
:1021F90036A20B4006E5412464F536E536D39464EE
:102209004009E536C39464F53680037536009000BD
:10221900BFE0C3953650069000BFE0F53622D200E4
:10222900900079E0A852B800049553504190007984
:10223900E0A852B800049553500375360F90007901
:10224900E004A852B800049553500375360A90006B
:1022590079E02402A852B800049553500575360553
:10226900C200900079E060067409900050F0C23A0B
:102279007E017F009000C5E01269089000D4E08ECD
:10228900048F05FF1268F8E55FBC0017D39D401362
:102299009000CEE0B40204D23A8002C200740A90DF
:1022A9000050F09000C6E0C3956750159000D8E043
:1022B900A852B8000495535002C200740B90005004
:1022C900F0E567C39464501D90011EE0600D900114
:1022D9001EE0A852B80006955340028008C2007457
:1022E9000B900050F0A2004003753605900107E0FD
:1022F900B40114900108E0A852B80004955350079E
:10230900E55FC39560400280089000B0E0F5368033
:102319003A90008FE0B40306A22AB3B34002802B9F
:102329009007CFE0C39405A852B800049553500C08
:102339009000B0E0F536740C900050F09007CFE0B3
:10234900A852B8000495535002C20085366C90001B
:1023590081E02536FE90004FE075F01E84FC7F0079
:10236900EE2CF5362290004FE075F00584FF7E00D3
:102379008F3790004FE075F00584ADF07C008D3A01
:10238900753F05755A03755BD69000D2E01475F058
:102399000584FF7E00E537BE00039F5005120D6AD4
:1023A900800BE53790045712693AE0F537E5379025
:1023B90007CEF09007CEE0FE9000C1E0C39E500822
:1023C9009000C1E09007CEF022E56775F00A84FF1E
:1023D9007E0090058112692FE0F546E546D39464A5
:1023E9004010E546C3946475F00F84FF7E008F4664
:1023F90080037546009000A4E02546F5462290002A
:10240900BCE0C3940350269007BBE0FEA3E0FF7431
:1024190004120039E55F126908740F8E048F05FFF5
:102429001268F89007B9ECF0A3EDF080249007BB8F
:10243900E0FEA3E0FF7404120039E5611269087433
:102449000F8E048F05FF1268F89007B9ECF0A3ED21
:10245900F0900097E0B40262E56AC3944175F00513
:1024690084FF7E008F37E56A75F00584ADF07C0046
:102479008D3A753F05755A06755B14E537C3941790
:102489005005120D6A80069006A8E0F5379007B945
:10249900E0FEA3E0FF740A8E048F05FF1268F8E5D9
:1024A900378C068D07126908740A8E048F05FF128E
:1024B90068F89007B9ECF0A3EDF09007B9E0FEA336
:1024C900E0FF9007BFE0FCA3E0FDEDD39FEC9E4049
:1024D9000F9007BFE0F8A3E09007B9C8F0A3C8F0D0
:1024E900229006C8E090386BF8282873804C8553F1
:1024F9007380479000D4E0855FF0A4FFAEF07408C4
:102509001200398F738033856173802E85677380DC
:10251900298568738024856973801F856A73801A89
:10252900856B7380158566738010856573800B854F
:0A2539006C73800690001AE0F57341
:10386B000224F50224F70224FC022510022515027E
:10387B00251A02251F02252402252902252E0225A1
:07388B003302253802253D40
:102543009006C9E0FE9006CAE0D39E404B9006C8B1
:10255300E0B404189006CAE0C395735002D22B90DE
:1025630006C9E0D395734002C22B802A9006C9E0C6
:10257300C3957350099006CAE0D395735002800245
:10258300D22B9006C9E0D3957350099006CAE0C3D5
:1025930095735002C22B802A9006C9E0D3957340ED
:1025A300099006CAE0C3957340028002C22B9006CD
:1025B300C9E0C3957340099006CAE0D395734002FE
:1025C300D22B229006CCE0903892F8282873804CC6
:1025D30085537380479000D4E0855FF0A4FFAEF08D
:1025E30074081200398F738033856173802E856779
:1025F3007380298568738024856973801F856A7356
:10260300801A856B7380158566738010856573806A
:0C2613000B856C73800690001AE0F573D4
:103892000225D10225D30225D80225EC0225F10208
:1038A20025F60225FB02260002260502260A02262A
:0738B2000F02261402261983
:10261F009006CDE0FE9006CEE0D39E405F9006CCB4
:10262F00E0B404189006CEE0C395735002D22C90FC
:10263F0006CDE0D395734002C22C803E9006CDE0CC
:10264F00C3957350099006CEE0D395735002800264
:10265F00D22C9006CDE0D3957350099006CEE0C3EF
:10266F0095735002C22C9006CCE0B401099000E0A3
:10267F00E0D3956150028002C22C802A9006CDE0F3
:10268F00D3957340099006CEE0C395734002800244
:10269F00C22C9006CDE0C3957340099006CEE0D3CF
:1026AF0095734002D22C229006D0E09038B9F828CA
:1026BF002873804C85537380479000D4E0855FF07A
:1026CF00A4FFAEF074081200398F738033856173E5
:1026DF00802E856773802985687380248569738050
:1026EF001F856A73801A856B7380158566738010DA
:1026FF00856573800B856C73800690001AE0F57307
:1038B9000226C10226C30226C80226DC0226E1022C
:1038C90026E60226EB0226F00226F50226FA022651
:0738D900FF0227040227098A
:10270F009006D1E0FE9006D2E0D39E404B9006D0CB
:10271F00E0B404189006D2E0C395735002D22D9006
:10272F0006D1E0D395734002C22D802A9006D1E0E6
:10273F00C3957350099006D2E0D39573500280026F
:10274F00D22D9006D1E0D3957350099006D2E0C3F5
:10275F0095735002C22D802A9006D1E0D395734015
:10276F00099006D2E0C3957340028002C22D9006F5
:10277F00D1E0C3957340099006D2E0D39573400220
:10278F00D22D229006D4E09038E0F8282873804CA0
:10279F0085537380479000D4E0855FF0A4FFAEF0BF
:1027AF0074081200398F738033856173802E8567AB
:1027BF007380298568738024856973801F856A7388
:1027CF00801A856B7380158566738010856573809D
:0C27DF000B856C73800690001AE0F57307
:1038E00002279D02279F0227A40227B80227BD02B4
:1038F00027C20227C70227CC0227D10227D60227D8
:07390000DB0227E00227E5CE
:1027EB009006D5E0FE9006D6E0D39E404B9006D4E3
:1027FB00E0B404189006D6E0C395735002D22E9025
:10280B0006D5E0D395734002C22E802A9006D5E000
:10281B00C3957350099006D6E0D39573500280028E
:10282B00D22E9006D5E0D3957350099006D6E0C30F
:10283B0095735002C22E802A9006D5E0D395734033
:10284B00099006D6E0C3957340028002C22E900613
:10285B00D5E0C3957340099006D6E0D3957340023B
:10286B00D22E229006D8E0903907F8282873804C96
:10287B0085537380479000D4E0855FF0A4FFAEF0E2
:10288B0074081200398F738033856173802E8567CE
:10289B007380298568738024856973801F856A73AB
:1028AB00801A856B738015856673801085657380C0
:0C28BB000B856C73800690001AE0F5732A
:1039070002287902287B022880022894022899023B
:10391700289E0228A30228A80228AD0228B202285E
:07392700B70228BC0228C111
:1028C7009006D9E0FE9006DAE0D39E404B9006D8FA
:1028D700E0B404189006DAE0C395735002D22F9043
:1028E70006D9E0D395734002C22F802A9006D9E01B
:1028F700C3957350099006DAE0D3957350028002AE
:10290700D22F9006D9E0D3957350099006DAE0C329
:1029170095735002C22F802A9006D9E0D395734051
:10292700099006DAE0C3957340028002C22F900631
:10293700D9E0C3957340099006DAE0D39573400256
:10294700D22F229006DCE090392EF8282873804C8D
:1029570085537380479000D4E0855FF0A4FFAEF005
:1029670074081200398F738033856173802E8567F1
:102977007380298568738024856973801F856A73CE
:10298700801A856B738015856673801085657380E3
:0C2997000B856C73800690001AE0F5734D
:10392E0002295502295702295C02297002297502C3
:10393E00297A02297F02298402298902298E0229E5
:07394E009302299802299D54
:1029A3009006DDE0FE9006DEE0D39E404B9006DC11
:1029B300E0B404189006DEE0C395735002D2309061
:1029C30006DDE0D395734002C230802A9006DDE035
:1029D300C3957350099006DEE0D3957350028002CD
:1029E300D2309006DDE0D3957350099006DEE0C344
:1029F30095735002C230802A9006DDE0D395734070
:102A0300099006DEE0C3957340028002C23090064F
:102A1300DDE0C3957340099006DEE0D39573400271
:102A2300D230229006E0E0903955F8282873804C84
:102A330085537380479000D4E0855FF0A4FFAEF028
:102A430074081200398F738033856173802E856714
:102A53007380298568738024856973801F856A73F1
:102A6300801A856B73801585667380108565738006
:0C2A73000B856C73800690001AE0F57370
:10395500022A31022A33022A38022A4C022A51024B
:103965002A56022A5B022A60022A65022A6A022A6C
:073975006F022A74022A7997
:102A7F009006E1E0FE9006E2E0D39E404B9006E028
:102A8F00E0B404189006E2E0C395735002D231907F
:102A9F0006E1E0D395734002C231802A9006E1E04F
:102AAF00C3957350099006E2E0D3957350028002EC
:102ABF00D2319006E1E0D3957350099006E2E0C35E
:102ACF0095735002C231802A9006E1E0D39573408E
:102ADF00099006E2E0C3957340028002C23190066E
:102AEF00E1E0C3957340099006E2E0D3957340028D
:102AFF00D231229006E4E090397CF8282873804C7C
:102B0F0085537380479000D4E0855FF0A4FFAEF04B
:102B1F0074081200398F738033856173802E856737
:102B2F007380298568738024856973801F856A7314
:102B3F00801A856B73801585667380108565738029
:0C2B4F000B856C73800690001AE0F57393
:10397C00022B0D022B0F022B14022B28022B2D02D3
:10398C002B32022B37022B3C022B41022B46022BF3
:07399C004B022B50022B55DA
:102B5B009006E5E0FE9006E6E0D39E404B9006E43F
:102B6B00E0B404189006E6E0C395735002D232909D
:102B7B0006E5E0D395734002C232802A9006E5E069
:102B8B00C3957350099006E6E0D39573500280020B
:102B9B00D2329006E5E0D3957350099006E6E0C378
:102BAB0095735002C232802A9006E5E0D3957340AC
:102BBB00099006E6E0C3957340028002C23290068C
:102BCB00E5E0C3957340099006E6E0D395734002A8
:102BDB00D232229006E8E09039A3F8282873804C73
:102BEB0085537380479000D4E0855FF0A4FFAEF06F
:102BFB0074081200398F738033856173802E85675B
:102C0B007380298568738024856973801F856A7337
:102C1B00801A856B7380158566738010856573804C
:0C2C2B000B856C73800690001AE0F573B6
:1039A300022BE9022BEB022BF0022C04022C09025E
:1039B3002C0E022C13022C18022C1D022C22022C7A
:0739C30027022C2C022C311D
:102C37009006E9E0FE9006EAE0D39E404B9006E856
:102C4700E0B404189006EAE0C395735002D23390BB
:102C570006E9E0D395734002C233802A9006E9E083
:102C6700C3957350099006EAE0D39573500280022A
:102C7700D2339006E9E0D3957350099006EAE0C392
:102C870095735002C233802A9006E9E0D3957340CA
:102C9700099006EAE0C3957340028002C2339006AA
:102CA700E9E0C3957340099006EAE0D395734002C3
:102CB700D233229006ECE09039CAF8282873804C6A
:102CC70085537380479000D4E0855FF0A4FFAEF092
:102CD70074081200398F738033856173802E85677E
:102CE7007380298568738024856973801F856A735B
:102CF700801A856B73801585667380108565738070
:0C2D07000B856C73800690001AE0F573D9
:1039CA00022CC5022CC7022CCC022CE0022CE502E8
:1039DA002CEA022CEF022CF4022CF9022CFE022D06
:0739EA0003022D08022D0D60
:102D13009006EDE0FE9006EEE0D39E404B9006EC6D
:102D2300E0B404189006EEE0C395735002D23490D9
:102D330006EDE0D395734002C234802A9006EDE09D
:102D4300C3957350099006EEE0D395735002800249
:102D5300D2349006EDE0D3957350099006EEE0C3AC
:102D630095735002C234802A9006EDE0D3957340E8
:102D7300099006EEE0C3957340028002C2349006C8
:102D8300EDE0C3957340099006EEE0D395734002DE
:102D9300D23422AE2EAF2F74F5D39F74019E400818
:102DA300782E12695C022EB0752F01752E00AE527B
:102DB300AF53E546BE000DD39F40099000B6E0D364
:102DC300954740028023754700E546C39553F57345
:102DD3009000B9E0D395454008E5452573F5458056
:102DE300069000B9E0F54580020547900092E0D3D4
:102DF3009561401CE55FC395604015AE52AF53E546
:102E030046BE00039F50099000B7E0D395484002A7
:102E1300806E9007D2E0A852B80004955350037512
:102E23004A009007D2E0A852B8000BD3955340064E
:102E3300E5539007D2F0E54A7041E553C39546F553
:102E430073E573D3940540037573059000B8E0C32D
:102E530095455007E573C3954540028009E545C391
:102E63009573F54580069000B8E0F5459000B8E00D
:102E7300D3954540069000B8E0F5457548008002BB
:102E83000548E54A7016900092E0C39561500DE540
:102E9300462405A852B8000695534002800F9000BF
:102EA300A5E0F545754A0174789007D2F022AE2E5D
:102EB300AF2F74E9D39F74039E4008782E12695C88
:102EC30002304F752F01752E00754532A235402A09
:102ED3007545199000A5E075F002A4FFAEF0E54733
:102EE300BE0006D39F4002D2350547754A03747866
:102EF3009007D2F075490002303EAE52AF53E5461B
:102F03006F4E700302303EE546BE000DD39F40096D
:102F13009000B6E0D395474002800F754700E54A1D
:102F2300C394035003754519800DE546C39553F5C6
:102F330073E5472573F547900092E0D39561400E02
:102F43009007D2E0A852B80007D395534002800CF3
:102F530005499000A5E0B54903754A00E54AB40365
:102F630006A20BB3B34002800A0549E549B43C030A
:102F7300754A02E54AB402299007D2E0A852B80084
:102F83000ED395534009E5539007D2F0754900904D
:102F93000092E0C39561500975490074789007D297
:102FA300F0E54A705A900092E0D39561401CE55FCA
:102FB300C395604015AE52AF53E546BE00039F5024
:102FC300099000B7E0D39548400280087548007522
:102FD300454B8028E553C39546F573E573D39405B4
:102FE3004003757305900092E0D395614008E5486E
:102FF3002573F5488006E5482406F548754900E53C
:103003004A7016900092E0C39561500DE546240581
:10301300A852B80006955340028003754A01E54A59
:10302300B4011875451905499000A5E0B549067521
:103033004A0275490074789007D2F0E54575F00AA5
:10304300A4FFAEF09007C3EEF0A3EFF022E56F907C
:1030530039F1F828287390008AE0700302327790E0
:1030630000C0E0B40102800302319290004DE0B54C
:103073005E02800302318F7E017F00E5BE12690884
:10308300E5BD2FFF50010E8E5A8F5B741012690835
:10309300900078E08E048F05FF1268F89007C7EC64
:1030A300F0A3EDF074FFBC00039D500B74FF900779
:1030B300C7F8E4F0E8A3F0E56B600FE56BC394FE9B
:1030C30050089000E6E06402600280649000D4E05F
:1030D300B40B1F9007C7E0FEA3E0FF74E712690873
:1030E300E56B8E048F05FF1268F89007C7ECF0A319
:1030F300EDF09000D4E0D3940B40089000BCE06462
:10310300046002802B9007C7E0FEA3E0FF9007C98D
:10311300E0FCA3E0FDEFD39DEE9C400D12695490BB
:1031230007C7EEF0A3EFF080079007C7E4F0A3F022
:1031330090008AE0B4021E9007C7E0FEA3E0FF9070
:1031430007D3E02FFF50010E74011200399007C717
:10315300EEF0A3EFF09007C7E0FEA3E0FF9007D3E4
:10316300E0BE0008D39F4004D2388002B2389007F3
:10317300C8E09007D3F09000BCE064016006A23879
:10318300B3B3400280069007C8E0F55F023275D200
:10319300387E017F00E5BE126908E5BD2FFF5001AF
:1031A3000E8E5A8F5B7410126908900078E08E04BB
:1031B3008F05FF1268F89007C7ECF0A3EDF0E56BFD
:1031C300600FE56BC394FE50089000E6E064026074
:1031D3000280649000D4E0B40B1F9007C7E0FEA305
:1031E300E0FF74E7126908E56B8E048F05FF126830
:1031F300F89007C7ECF0A3EDF09000D4E0D3940B64
:1032030040089000BCE064046002802B9007C7E094
:10321300FEA3E0FF9007C9E0FCA3E0FDEFD39DEE22
:103223009C400D1269549007C7EEF0A3EFF080079E
:103233009007C7E4F0A3F090008AE0B4021E900761
:10324300C7E0FEA3E0FF9007D3E02FFF50010E7409
:10325300011200399007C7EEF0A3EFF09007C8E022
:103263009007D3F09000BCE0640160069007C8E0CB
:10327300F55F8003755F00900086E07006756F014F
:1032830002305075BB18023845900086E070030287
:1032930033FD7E017F00E5BE126908E5BD2FFF50B7
:1032A300010E8E5A8F5B9000CCE0B4010F7E0F7F2E
:1032B300FFAC5AAD5B1269548E5A8F5B9000F1E0FC
:1032C300B40245AE5AAF5B900023E0FCA3E0FDEDF2
:1032D300D39FEC9E400A900023E55AF0A3E55BF0F0
:1032E300AE5AAF5B900025E0FCA3E0FDEFD39DEE6B
:1032F3009C400A900025E55AF0A3E55BF0AE5AAF77
:103303005B74041200398F619000F1E0704CAE5A87
:10331300AF5B900023E0FCA3E0FDEFD39DEE9C4068
:10332300091269548E5A8F5B8006755B00755A00CB
:10333300AE5AAF5B7410126908900075E08E048F6B
:1033430005FF1268F88C5A8D5B74FFBC0009D39D8E
:103353004005855B6180037561FE9000BCE0B401AC
:103363000280030233FBA20BB3B3500E900090E034
:10337300A852B80005D39553500280719000CDE058
:103383008561F0A4FFAEF074648E048F05FF1268AC
:10339300F88C5A8D5BE56B6016E56BC394FE500F9A
:1033A3009000E6E0B402089000D4E0640B60028071
:1033B30017AE5AAF5B74E7126908E56B8E048F058D
:1033C300FF1268F88C5A8D5BAE5AAF5B9007C7E06B
:1033D300FCA3E0FDEDD39FEC9E4005855B5F800B76
:1033E300A238B340069007C8E0F55F800BA238B35C
:1033F30040069007C8E0F55F80037561009000897F
:10340300E07006756F0202305075BB1902384590A3
:103413000089E070030234B2E55ED39551400302A4
:1034230034B0900021E0FEA3E0FFE56512694C9003
:103433000021EEF0A3EFF07E017F00E5BE126908E4
:10344300E5BD2FFF50010E8E5A8F5B9000F6E070A2
:1034530013740A12690874518E048F05FF1268F8F9
:103463008D658019AE5AAF5B740A1269088F048E9A
:10347300057E017F95CDCCCD1267F68F65E565D3CB
:1034830094644003756564900021E0FEA3E0FFE5CA
:10349300652FFF50010E900021EEF0A3EFF0900096
:1034A3008DE0048E048F05FF1268F88D6580037527
:1034B30065329000D9E07006756F0302305075BB1A
:1034C300130238459000D9E0604A7E017F00E5BED3
:1034D300126908E5BD2FFF50010E8E5A8F5B7404ED
:1034E3001200398F669000DBE08566F0A4FDACF036
:1034F3007464FF1268F88D669000DAE08566F0A4C4
:10350300FFAEF074FF8E048F05FF1268F8ED900094
:1035130074F08003756600900087E07006756F0491
:1035230002305075BB17023845900087E0B40102A2
:1035330080030235C07E017F00E5BE126908E5BD48
:103543002FFF50010E8E5A8F5B9007D4E0601990C5
:1035530007D4E01490638212008CE493FC7401930B
:10356300FDEDC39FEC9E400280069007D4E014F06B
:103573009007D4E0C394B3501DAE5AAF5B9007D409
:10358300E00490638212008CE493FC740193FDEFDA
:10359300C39DEE9C400280069007D4E004F09007A0
:1035A300D4E0FE9000ADE08E0088F0A4FFAEF0748E
:1035B300648E048F05FF1268F88D678003756700BA
:1035C300900088E07006756F0502305075BB1602D7
:1035D3003845900088E0B4010280030236697E0119
:1035E3007F00E5BE126908E5BD2FFF50010E8E5A1C
:1035F3008F5B9007D5E060199007D5E0149064ECD9
:1036030012008CE493FC740193FDEDC39FEC9E4088
:103613000280069007D5E014F09007D5E0C394B379
:10362300501DAE5AAF5B9007D5E0049064EC1200D6
:103633008CE493FC740193FDEFC39DEE9C400280E8
:10364300069007D5E004F09007D5E0FE9000B3E0C4
:103653008E0088F0A4FFAEF074648E048F05FF1211
:1036630068F88D68800375680075BB1F0238457E56
:10367300017F00E5BE126908E5BD2FFF50010E8EE4
:103683005A8F5B740912690874E68E048F05FF1262
:1036930068F88D6A90008FE07006756F07023050EE
:1036A30075BB1502384590008FE070030237C47E66
:1036B300017F00E5BE126908E5BD2FFF50010E8EA4
:1036C3005A8F5B74041200398F6990008FE0B40144
:1036D300159000E3E08569F0A4FFAEF074071200D3
:1036E30039EF9007CCF090008FE0B402159000E31F
:1036F300E08569F0A4FFAEF07407120039EF90077C
:10370300CBF090008FE0B4030280030237A7900050
:10371300D0E0701CE569C394195002D22AE569D33D
:1037230094644002C22A9000AFE09007CFF0806318
:103733009000AFE070349000E3E08569F0A4FFAE41
:10374300F074FF8E048F05FF1268F8ED9007CFF039
:10375300AE52AF53741EBE0006D39F4002D22AE579
:1037630061D394E54002C22A8029E569C3940A50D3
:103773000DAE52AF53741EBE0004D39F500280029D
:10378300D22AE561D394E54002C22A9000AFE090CB
:1037930007CFF09007CFE0C3940550067405900758
:1037A300CFF0C23990008FE0B40414E569C39419D3
:1037B3005002D239E569D394324002C239C22A8019
:1037C300037569009000E6E07006756F08023050DB
:1037D30075BB14806D9000E6E060567E017F00E5C6
:1037E300BE126908E5BD2FFF50010E8E5A8F5BEFA5
:1037F300D39421EE940E4005756BFF8015AE5AAF3E
:103803005B741012690874E38E048F05FF1268F865
:103813008D6BE56B75F00BA4FFAEF09000D4E08EDA
:10382300048F05FF1268F89007C9ECF0A3EDF08050
:1038330003756B0090008AE0600575BB1A80037501
:02384300BB18B0
:1039F10002305902328C0234120234C702352C02D1
:0B3A010035D50236720236A90237D814
:05384500056FD2EC222A
:09693A002582F58250020583223A
:0F008C0025E050020583258250020583F582226C
:1068D700EF2F500205832582F582E5833E2EF5834F
:0168E700228E
:10694C00CFC39FFF50011E22C3EF9DFFEE9CFE2282
:08695C000806B600021806222D
:0D691600A3E004F07006120049E004F02236
:0E003900048007C3CE13CECF13CFD5E0F6223E
:1067F600BC000FBE0008ED8FF084FFADF022E4FE72
:10680600FF22BE000DEF60FE54F0606F20E703022A
:1068160068ACEAC0E0EBC0E078017A0075F001EE02
:1068260020E710EF25E0FFEE33FE0AC5F023C5F0A2
:1068360030E7F0EA5407F9096A7A007B006001083C
:10684600C3EC9E40167004ED9F4010ED9FFDEC9E3C
:10685600FCE5F0CA4ACA03F5F08005E5F003F5F059
:10686600C3EE13FEEF13FFD9D77908CACBCAD8D027
:10687600EAFEEBFFD0E0FBD0E0FA22EC8FF084FCDE
:10688600ED54F045F0C48FF084FEEDC454F045F0AD
:10689600C48FF084FDEEC4FE54F02DFFEE540F3C81
:1068A600FEADF07C0022790078008FF0EC7E0820A7
:1068B600E70DC3CD33CD33C933C9C833C8DEF08441
:1068C60049F9E5F08FF0BE00E6FD7C00E9FFE8FE41
:0168D600229F
:0E690800F88FF0A4FFE5F0CE88F0A42EFE225A
:10000300EF8DF0A4F9A8F0EF8CF0A428F8EE8DF0B2
:06001300A428FEE9FF2213
:1068E800600D782B0268F2007830D8FED5E0F822E7
:1068F800EEC0E07E001267F6EFFDEEFCD0E0FE226F
:0C692300EEC0E07E001267F6D0E0FE221D
:03001B0002001EC2
:0300530002005652
:03009B00020071EF
:030000000269434F
:0969430075817575D00002445302
:0B692F00E5822FF582E5833EF5832210
:0A0049000582D5820215831582227C
:10001E00C0E0C0F0C083C082C0D075D0001243BF14
:0B002E00D0D0D082D083D0F0D0E032E0
:10005600C0E0C0F0C083C082C0D075D0001243C2D9
:10006600D0D0D082D083D0F0D0E032C0E0C0F0C093
:1000760083C082C0D075D0001243DED0D0D082D0EB
:0600860083D0F0D0E0324F
:00000001FF
